:020000040800F2
:1000000000500020359B0008319B00082F9B000802
:100010002F9B00082F9B00082F9B0008000000006A
:10002000000000000000000000000000319B0008FC
:10003000319B000800000000319B0008319B000844
:100040002F9B00082F9B00082F9B00082F9B000868
:100050002F9B00082F9B00082F9B00082F9B000858
:100060002F9B00082F9B00082F9B00082F9B000848
:100070002F9B00082F9B00082F9B00082F9B000838
:100080002F9B00082F9B00082F9B00082F9B000828
:100090002F9B00082F9B00082F9B00082F9B000818
:1000A0002F9B00082F9B00082F9B00082F9B000808
:1000B0002F9B00082F9B00082F9B00082F9B0008F8
:1000C0002F9B00082F9B00082F9B00082F9B0008E8
:1000D0002F9B00082F9B00082F9B00082F9B0008D8
:1000E0002F9B00082F9B00082F9B00082F9B0008C8
:1000F0002F9B00082F9B00082F9B00082F9B0008B8
:100100002F9B00082F9B00082F9B00082F9B0008A7
:100110002F9B00082F9B00082F9B00082F9B000897
:100120002F9B00082F9B00082F9B00082F9B000887
:100130002F9B00082F9B00082F9B00082F9B000877
:100140002F9B00082F9B00082F9B00082F9B000867
:1001500061B6704771B670472DE9F843364801F033
:1001600021FB4FF0E023D3F8002D3448D3F8005D95
:10017000D3F8004DD3F8007DD3F8006DD3F8001DFF
:100180004FEA1268DFF8B89001F026FA2D4942468E
:10019000B8F1410F18BF49462B4801F01DFAC5F3CD
:1001A00003452A4801F018FA0C2DC4F30B14C7F3C9
:1001B000035706F00F0603D00F2D1CD0484600E071
:1001C000234801F009FA2946224801F005FA22489D
:1001D00001F002FA40F627439C420ED8B4F5426F74
:1001E00027D3A4F54263072B23D8DFE803F01A22B4
:1001F000221C1E2222201948E3E7B4F5466F18D1CD
:10020000174801F0E9F92146164801F0E5F93946A9
:10021000154801F0E1F93146BDE8F843134801F013
:10022000DBB91348EDE71348EBE71348E9E7134858
:10023000E7E70348E5E700BF1CA500082EA5000876
:1002400014A5000810A5000841A500085EA5000837
:100250006FA500087FA5000889A5000877A50008FC
:1002600099A50008CCA50008D8A50008E8A50008B5
:10027000A4A50008AEA50008B8A50008C2A50008FE
:1002800038B5184C184801F08DFA226823681748D1
:1002900021681B0CC2F30B0201F09EF94FF0E02322
:1002A000D3F8F05D124B15F001051249124808BF52
:1002B000194601F091F97DB140F2073322689A4264
:1002C00004D10E48BDE8384001F06CBA23680BB980
:1002D0000B48F7E70B48F5E723680BB90A48F1E745
:1002E0000A48EFE7002004E000A600082BA600085B
:1002F000FDA50008F9A5000862A6000879A6000877
:10030000D2A6000835A70008A6A70008FDA7000888
:100310001D4A70B5D2F8E45FD2F8E84FD2F8D06F3A
:10032000C5F3031192F8E03F24012D0206F00F06F9
:1003300004F0700405F4706514480C431D4301F08B
:100340004BF966B9202C1CD1114801F045F92B4618
:1003500022463146BDE870400E4801F03DB9072EF7
:1003600003D1512C0DD10C48EFE7042E03D13B2CC7
:1003700007D10A48E9E7052E03D1552C01D10848D9
:10038000E3E70848E1E700BF00F00FE04BA80008F2
:1003900057A800086EA800085BA8000810A5000870
:1003A00066A8000814A500082DE9F04F0025ADF55A
:1003B0002F7D664801F0F6F94FF0E023A846AA46E3
:1003C0002C46FFF7C7FED3F8282DDFF884B142F49E
:1003D0000042C3F8282DD3F8142D42F48072C3F8DC
:1003E000142DD3F8286D86F40046C6F3C0362B785A
:1003F0004FF0E023D3F8287DB14607F40047002FE3
:100400000FBF01260026D3F8282D42F4004218BF62
:10041000C3F8282D4E4530D04FF0E022D2F8143DDD
:100420004C4923F48073C2F8143D4B4B6A1EB9F15A
:10043000000F08BF0B4658465146FFF789FE019250
:1004400001F0CAF8382C0DD80C2363430DF10C0CC5
:10045000019A0CEB030001344CF803A0426080F8D1
:100460000890E4B24FF0E022AA46FFF773FED2F8FC
:10047000143D43F48073C2F8143D15F5807548F1BE
:100480000008B8F1010F08BF002DB0D14FF0E022F5
:10049000D2F8143D514623F48073C2F8143D2E4A1D
:1004A0002C4B2B48002F08BF13464FF0FF32FFF7AD
:1004B0004FFE01F091F8382C0BD80C23634303A8AE
:1004C000C21840F803A04FF0FF3301345360167296
:1004D000E4B20026B646214D214F95F80880A0458C
:1004E00020D10023D5F804C003AADCF8000011686D
:1004F000884217D1DCF804005168884212D19CF878
:100500000800117A88420DD10133DBB298450CF115
:100510000C0C02F10C02E8D13846296801F05CF8B5
:100520004FF0010E03360F2E05F10C05D5D1BEF1AB
:10053000000F06D10B480DF52F7DBDE8F04F01F0FF
:1005400031B90DF52F7DBDE8F08F00BFA1A80008DF
:10055000DCA8000894A8000896A8000890B5000838
:1005600050A90008F4A80008304B2DE9F041D3F859
:10057000E84FD3F8D05FD3F8E43F2401C3F303136B
:1005800004F070041C434FF0E0232948D3F8008D99
:10059000D3F8007DD3F8006D01F01EF840F6234338
:1005A000C8F30B18984505F00F05224BC7F3035706
:1005B00006F00F0611D1012F0FD1012E32D1002DDF
:1005C00030D1202C2ED11C4A1C481A6001F004F8AE
:1005D000BDE8F0411A4801F0E5B8022F22D1012E02
:1005E00020D1072D05D1512C1CD1164A16481A606E
:1005F000ECE7042D0ED13B2C14D1144A1268C2F33F
:100600000B021AB1124A13481A60DFE7124A134864
:100610001A60DBE7052D05D1552C03D1104A11488E
:100620001A60D3E7104A11481A60CFE700F00FE0D4
:100630006AA900080C00002057A8000879A9000842
:10064000CDB000088CA900085BA80008002004E0D9
:100650008FA9000893A90008A4A90008A8A9000868
:10066000AFA90008B2A90008BBA9000814A500089A
:1006700070B5094801F096F80025084C084E21682D
:10068000626830460B68013500F0A6FF132D04F1B7
:100690000804F4D170BD00BFBFA9000894C10008D0
:1006A000D3A9000807B50948D0F8F017D0F8EC270F
:1006B000D0F8E837D0F8E8079BB2000C0090044867
:1006C00000F08AFF03B05DF804FB00BF00F0FF1FDD
:1006D000EDA900082DE9D841A84BA9481E681F685C
:1006E000C6F30B0603F53D23D3F8E44FD3F8E08FB0
:1006F00000F072FF1EB140F207339E421BD124026C
:1007000004F470645FFA88F844EA080421469D48BE
:1007100000F062FF40F233439C4261D8B4F5826F2F
:100720000FD2002C00F08E8040F207339C4200F084
:10073000B280954887E03146944800F04DFF34463A
:10074000E8E7A4F58264232CF3D801A353F824F03E
:10075000A5080008330700089B08000809090008DD
:10076000AF08000833070008330700083307000804
:10077000C3080008130900083307000833070008FE
:100780003307000833070008330700083307000861
:100790003B09000833070008330700081D0900085B
:1007A0003307000833070008330700083307000841
:1007B000450900083307000833070008330700081D
:1007C0003307000833070008330700083307000821
:1007D000B908000831090008330700082709000894
:1007E000B4F5896F1CD8B4F5886FA2D3A4F58864DA
:1007F000082C9ED801A353F824F000BFE10800089C
:1008000033070008F508000833070008CD08000882
:10081000D70800083307000833070008EB08000872
:1008200040F266439C426AD040F2C3439C4200F0CF
:100830008E80B4F58C6F7FF47CAF554B554A56488B
:100840001A6000E0554800F0C7FE554800F0AAFFC6
:10085000002E00F01A8140F207339E4200F015810D
:100860003C0C21464F4800F0B7FEB6F5836F274693
:1008700072D8B6F5826F73D3A6F58266082E6FD84C
:10088000DFE816F0D2006E0070006E00E7006E0028
:100890006E006E00F9004448D5E73D4B434A44489A
:1008A0001A60D0E73A4B414A42481A60CBE7384BCE
:1008B0003E4A41481A60C6E7354B3C4A3F481A60F9
:1008C000C1E7334B394A3E481A60BCE7304B3D4ADA
:1008D0003D481A60B7E72E4B3C4A3D481A60B2E7E4
:1008E0002B4B3C4A3C481A60ADE7294B3B4A3C48FD
:1008F0001A60A8E7264B3B4A3B481A60A3E7244B03
:100900003A4A3B481A609EE7214B3A4A3A481A60F5
:1009100099E71F4B394A3A481A6094E71C4B394A09
:1009200039481A608FE71A4B364A38481A608AE706
:10093000174B374A37481A6085E7154B364A374810
:100940001A6080E7124B344A35481A607BE7104B37
:10095000164A34481A6076E7B6F5866F00F085804F
:10096000094873E0B4F5805FFAD1412000F04CFEF5
:100970000B48BDE8D84100F015BF00BF002004E0DF
:1009800016AA000823AA000814A500083AAA00081D
:100990000400002041AB00084AAB00084CAA000844
:1009A000CDB0000850AC000874AA00084BAC000899
:1009B0009DAA0008B3AA0008CCAA0008E3AA000870
:1009C000F8AA000814AB00080FAB00081EAB000823
:1009D00019AB000828AB000823AB000832AB0008B5
:1009E0002DAB00083CAB000837AB000862AB000839
:1009F0006BAB000883AB000894AB0008BCAB0008ED
:100A0000C5AB0008D9AB0008DEAB0008ECAB0008B2
:100A1000FAAB0008FFAB00080DAC000812AC0008F0
:100A20002FAC000846AC0008002C9ED0B4F5005F47
:100A300001D142209AE742F201039C4201D15A209F
:100A400094E742F203039F428AD1114800F0C4FDAB
:100A50008EE7B4F5805F01D10E48F7E741F201035C
:100A60009C42ECD041F20303EDE741F203039C42C8
:100A70007FF476AFF0E7B4F5805F3FF476AF41F2F4
:100A800001039C427FF46CAFD9E7034871E700BFD4
:100A900070AC00087AAC00087EAC00082DE9F04F7D
:100AA000DFF8AC916B4887B000F07CFE4FF0000A95
:100AB000CB464FF0E02600234FF0010801938CE075
:100AC000FFF748FBD6F8283D43F40043C6F8283D1D
:100AD000D6F8143D43F48073C6F8143D2301039304
:100AE000D9F8043003EB0414029363681B68D6F84A
:100AF000283D13F4004F18BF4FF00008D6F8283DEA
:100B000043F40043C6F8283DD6F8143D23F480731F
:100B1000C6F8143DFFF71CFBB8F1000F00F0818010
:100B2000DDE90232985A08F001FF002300939DF896
:100B30000070237BBB4201D8454645E00023059366
:100B4000059B092B17D9A3680222002133F817301F
:100B5000606808F071FEA368606833F8171008F049
:100B6000B7FEA368606833F8171008F0B4FE28B128
:100B7000009B0133DAE7059B0133E0E7A368606877
:100B800033F8171008F0A2FE6068A268C36832F854
:100B9000171085680D4003D00B4214BF01250025B6
:100BA00008F096FE6068A368C26833F81730002129
:100BB0001A42826818BF0025134218BF002501227F
:100BC00008F03AFE002DD3D1A846DDE90232985A4A
:100BD00008F0ACFE019B0133019399F808309DF8B1
:100BE0000440A3423FF66CAFB8F1000F19D00C23BC
:100BF00003FB0AFA0BEB0A035C781BF80A50224647
:100C00002946154800F0E8FC144B1D70144B1C706D
:100C1000134B1B78CBB9134807B0BDE8F04F00F079
:100C2000C1BD0C2303FB0AF30BEB030252781BF844
:100C300003100D480AF1010A00F0CEFCBAF1050FCD
:100C400009F10C097FF437AFE2E707B0BDE8F08F98
:100C5000DCB80008AEAC000805AD000810000020AC
:100C6000E309002067AD000834AD00082DE9F74F17
:100C7000424800F097FD0026414C424FDFF808A1A2
:100C80000022D4E90251D4F80080B4F804B0B4F8DA
:100C90000690019107F8012BB8F1000F59D0002DF3
:100CA00057D0584608F042FE484608F05CFE4FF028
:100CB000E020FFF74FFAD0F8283D002243F400432C
:100CC000C0F8283DD0F8143D43F48073C0F8143DBB
:100CD000D5F800E0D0F8283DD0F828CD13F4004333
:100CE0004CF4004CC0F828CD44D12A6801990A433D
:100CF0002A602A68C5F800E0D0F8285D15F41F4F77
:100D00002FD131EA02030CBF0125002501234FF04A
:100D1000E021D1F8142D019322F48072C1F8142D32
:100D20004846FFF715FA08F01EFE584608F00CFE7C
:100D3000019B002B14BF2B46002307F8013C1BD05E
:100D4000124A134B002D18BF1A464146504600F078
:100D500043FC04366C2E04F1100491D103B0BDE8BD
:100D6000F08F1D46D0F8282D42F41F42C0F8282DE0
:100D70002B46CCE71546FBE7064AE6E7BAAD000886
:100D8000A4B60008C8090020D8AD0008B3AD00081B
:100D9000ABAD0008A3AD000870B5214800F01CFC05
:100DA000204A13685B0C5B04B3F1005F33D15468D5
:100DB00024F47F6424F00F0494422CD140F2862066
:100DC00008F0B4FD08F088FB174E54F8040B08F047
:100DD0008BFBB4420546F8D1144B98420BD1144812
:100DE00000F0FAFB2946134800F0F6FBBDE870401E
:100DF000114800F0D7BC114B984201D11048EFE7E1
:100E0000104B984201D11048EAE7104B98420CBFB2
:100E10000F481048E4E7104800F0DEFBE6E700BFAB
:100E2000E3AD000800F0FF1FE0F7FF1F3221998FAC
:100E3000F3AD00085CAE0008CDB00008AFB63803D3
:100E400009AE00082AF654AC1EAE000848C09691C0
:100E500034AE000849AE0008B3AD000808B508F08C
:100E600057FBFF280BD8074B1B685B0C5B04B3F1E7
:100E7000005F14BF4FF400604FF4806008BD4FF472
:100E80000060FBE700F0FF1F2DE9F041964800F0FD
:100E900089FC964800F0A0FB08F03AFB4FF6FF7380
:100EA000984240F0E880924800F07CFC4FF0E0254A
:100EB0004FF00064FFF74EF9D5F8283D43F40043A6
:100EC000C5F8283DD5F8143D43F48073C5F8143DAA
:100ED000D5F8283D1A0440F1D580D5F8283D04F115
:100EE000784143F40043C5F8283DD5F8143D013955
:100EF00023F48073C5F8143D8A0A7E48FFF728F969
:100F000000F06AFB08F004FB0146002853D0FFF70D
:100F100021F9D5F8283D4FF0E02743F40043C5F808
:100F2000283DD5F8143D42F2423843F48073C5F8A9
:100F3000143D08F00FFC08F0EBFA810201F10065A6
:100F40002C466D4E2368D7F8283D1B041ED420463E
:100F500008F0A2FB08F05EFB202817D142F24231D4
:100F6000204608F067FB08F055FB20280ED12388A7
:100F700043450BD1204608F08FFB08F04BFB20289F
:100F800004D1FFF76BFF0444B442DBD308F02CFB21
:100F900008F0ECFB4FF0E023D3F8282D611B42F45E
:100FA0000042C3F8282DD3F8142D22F48072C3F820
:100FB000142DFFF7CDF88A0A504800F00DFB4FF0D2
:100FC000E0224FF00054FFF7C5F8D2F8283D214643
:100FD00043F40043C2F8283DD2F8143D422543F4BF
:100FE0008073C2F8143D23461878D2F8286DC0B239
:100FF000360410D41D70D2F8281D090404D41978C1
:10100000422904BF1C461870581CB0F1085F1946ED
:101010003DD16FF05E414FF0E023D3F8282D01F170
:10102000604142F40042C3F8282DD3F8142D013159
:1010300022F48072C3F8142D31488A0AFFF788F829
:1010400000F0CAFA04F1604101318C0A22462D48B1
:1010500000F0C2FA2C4B1C7008F05AFAB0F5807FF1
:1010600039D01BD8402833D013D8102829D02028B5
:101070002BD0BDE8F08108F04BFA0146234800F080
:10108000ABFA13E72378FFF7E9FE044420E70346B1
:10109000AAE78028EDD142221D4B14E0B0F5407F35
:1010A0001FD008D8B0F5C07F18D0B0F5007FE0D1D0
:1010B0004522174B07E0B0F5806FDAD14722144B79
:1010C00001E03422124B1A70D3E73622104BFAE7B4
:1010D00038220F4BF7E743220D4BF4E744220C4B29
:1010E000F1E746220A4BEEE76BAE0008A0AE00081F
:1010F000BAAE0008FEAE0008FFEFFF1F2AAF0008DF
:1011000066AF00088CAF0008E4090020F6AE0008C6
:10111000080000202DE9F74F474D484800F05CFAE1
:101120004749286800F01EFC28B9464C2070FFF79C
:101130001BFA01232370444E4149306800F012FC31
:1011400028B9404C2070FFF7C5FA0123237034689A
:101150003E49204600F006FC28B120463C4900F0FC
:1011600001FC002865D100230127364CDFF8E4801C
:101170002370FFF77BFD98F8003027701BB92370B0
:10118000FFF782FE2770344F3B783F2B02D0334B62
:101190001B782BB900232370FFF780FC01232370F9
:1011A0002F4C4FF00009A2460EE012F801CF11F8C3
:1011B000010B93420DD08445F7D009F10109B9F133
:1011C000120F04F10C0421D0A36826495A1E1A33C9
:1011D000EBE78445F1D194F804B008F099F9834520
:1011E000EBD1627998F800309A42E6D11B4BA27994
:1011F0001B789A42E1D10C2303FB09F95AF8094004
:101200000F49204600F0AEFB296858B9164B3268EA
:101210001B78296800933B78144800F0DDF903B08F
:10122000BDE8F08F2246124803B0BDE8F04F00F051
:10123000D3B922462968F6E70C000020B2AF0008B7
:10124000BBA9000800000020040000204BAC0008EF
:101250000DAC0008E409002010000020E309002084
:10126000CCB50008C809002008000020E2AF000843
:10127000D9AF0008F8B50D4B0E461B7814467BB16C
:1012800001280FD000F092F905234FF0FF340360DE
:1012900006E0715D384608F0EEFB0135A542F8DB4B
:1012A0002046F8BD0025024FF8E700BF00000020EF
:1012B00000380140F8B540F2023008F037FB4FF437
:1012C000407008F033FB40F20E3008F02FFB4FF473
:1012D000007302220321964808F0AEFA4FF48061B1
:1012E000934808F0F3FA4FF48063022200219048FB
:1012F00008F0A2FA4FF4E1318E4808F07DFB082196
:101300008C4808F08DFB00218A4808F092FB0C21E4
:10131000884808F09AFB0021864808F090FB0021DD
:10132000844808F098FB834808F09BFB824B02221C
:10133000186800238068194600F03CFA7F4800F0E6
:1013400031FA7C4E7E4F7F4D304608F09FFBC4B291
:101350002146384600F040F9792C05D8602C05D894
:101360000A2CF1D00D2CEFD077486BE0613C182CA3
:10137000FAD801A353F824F007140008DD1300087D
:101380004B14000869130008511400085714000892
:1013900069130008691400085D140008631400084C
:1013A00069130008DF140008E5140008EB140008B6
:1013B00069130008F114000869130008F714000805
:1013C0000F150008151500081B1500082115000849
:1013D00069130008691300082B1500085B4800F02A
:1013E000E1F9544C4021204608F09BFB0028F9D03D
:1013F0004FF0E022564BC2F8083D1A6882F3088885
:101400005B689847FEE70121284600F0E5F8FFF702
:1014100049F9FEF7A1FEFEF77BFFFFF7A5F8FFF7FE
:1014200059F9FFF731FDFFF721FCFFF737FBFFF715
:1014300071FEFFF7B1FCFFF71BF9FEF721FFFEF786
:10144000B3FF444800F0AEF97EE7FEF785FE7BE788
:10145000FEF716FF78E7FFF73DF975E7FFF75AFE4D
:1014600072E7FEF755FF6FE73B4800F09BF93B48FA
:1014700000F098F93A4800F095F93A4800F092F9EE
:10148000394800F08FF9394800F08CF9384800F0FD
:1014900089F9384800F086F9374800F083F9374871
:1014A00000F080F9364800F07DF9364800F07AF90E
:1014B000354800F077F9354800F074F9344800F009
:1014C00071F9344800F06EF9334800F06BF9334895
:1014D00000F068F9324800F065F93248B2E7FEF7EB
:1014E00063FF31E7FFF740F82EE7FFF7D7FA2BE766
:1014F000FFF7BCFB28E72C4800F054F90D4C4021C5
:10150000204608F00EFB0028F9D008F065FBFFF735
:10151000BBFC19E7FFF7ACF816E7FFF7C3F813E7D2
:101520000121284600F058F80EE7FFF735FC0BE7DD
:10153000000801400038014014000020EFAF00080F
:10154000EAAF000832B00008B2B200080FB00008DD
:1015500000F0FF1F4BB0000855B000086AB000084B
:101560007FB00008A4B00008CFB00008EDB00008BC
:1015700008B1000820B1000836B1000855B10008D4
:1015800064B100087DB1000892B10008A7B100085D
:10159000C0B10008D9B10008F0B1000805B20008D8
:1015A0002FB2000841B20008A7B20008014B18682A
:1015B000704700BF140000200EB400B582B003AB2A
:1015C00053F8042B8168019300F0D8FA02B05DF85B
:1015D00004EB03B0704700BF0FB400B5074A83B0F7
:1015E00004AB106853F8042B8168019300F0C6FA2D
:1015F00003B05DF804EB04B0704700BF1400002096
:10160000826800F009B800BF024B01461868826882
:1016100000F002B81400002070B505460E461446CE
:1016200008B1836BEBB1636ED80702D4A389990527
:1016300023D5A368013B002BA3601CDAA269934267
:1016400012DBF0B20A280FD0054623685A1C22602C
:101650001E70636EDA0702D4A3899B0511D5284654
:1016600070BD03F079FADEE728462246314602F0E3
:101670006FF80546EDE7F0B2E6E7A06D03F0FCFE7B
:10168000D7E7A06D03F000FF284670BD1D4B70B575
:101690001E6805460C460EB1B36BEBB1636ED807FE
:1016A00002D4A389990524D5A368013B002BA3602C
:1016B0001DDAA269934213DBE8B20A2810D006466D
:1016C00023685A1C22601D70636EDA0702D4A38956
:1016D0009B0512D5304670BD304603F03DFADDE77C
:1016E00030462246294602F033F80646ECE7E8B2D7
:1016F000E5E7A06D03F0C0FED6E7A06D03F0C4FEE1
:10170000304670BD1400002030B5054689B008464B
:101710000C4600F005FA01210223214A04940692A6
:10172000AA6B04AC0590084401940791AC6802933D
:1017300003901AB3616EB4F90C30C9079AB201D4A0
:10174000900525D5910406D4626E43F4005322F42B
:101750000052A3816266284601AA214603F06EFC6E
:10176000636E002814BF4FF0FF350A25DA0702D454
:10177000A3899B0506D5284609B030BD284603F04D
:10178000EBF9D7E7A06D03F07FFE284609B030BD26
:10179000A06D03F071FEB4F90C309AB2D2E700BF2D
:1017A00030C20008024B01461868FFF7ADBF00BF0A
:1017B000140000202DE9F043694C0E46D4F8008057
:1017C000174604461D4683B0B8F1000F03D0D8F881
:1017D0003830002B77D0022F05D0012F00F2AC80DB
:1017E000002DC0F2A980636EDA0752D5214640462B
:1017F00003F006F9216B41B104F14003994202D094
:10180000404603F01FFB002323630023B4F90CC000
:10181000A3611CF0800F636064D12CF44A6C2CF03F
:10182000030C022FA4F80CC06AD001AB214640463D
:101830006A4603F09BFEA3891843A081002D2FD098
:10184000002E2ED0D8F83830002B38D0009AB4F9BA
:101850000C30AA421CBF43F40063A381012F04BFD4
:1018600043F00103A3819AB213F00803C4E90465AD
:1018700026602CD0D1075DD500216D42A561656E33
:10188000A16015F0010527D00025284603B0BDE86A
:10189000F083A3899B05A9D4A06D03F0EDFDA5E716
:1018A000009D284603F092FE0646002847D0A389F3
:1018B00043F08003A381D8F83830002BC6D14046CE
:1018C00003F04AF9C2E7404603F046F983E7A36014
:1018D000656E15F00105D7D1930524D5284603B0D0
:1018E000BDE8F0834046216903F0ACFAB4F90CC0BE
:1018F000022F2CF44A6C2CF0030CA4F80CC094D1E9
:1019000000250021012204F1430323602361636E5B
:101910004CF0020CD807A4F80CC0A1606261DDD4C1
:101920001CF4007FDAD1A06D03F0AEFD284603B0B1
:10193000BDE8F083A560CBE74FF0FF35CEE7DDF8DB
:101940000090A94504D0484603F040FE064620B961
:101950004FF0FF35B4F90CC0D3E74D46A7E700BF01
:101960001400002080EA010C1CF0030F37D110F0A6
:10197000030C20F0030021F0030150F8042B08BFF2
:1019800051F8043B0ED08CF0030C6FF07F434FEA0C
:10199000CC0C23FA0CFC51F8043B42EA0C0243EA5B
:1019A0000C0300BFA2F1013C9A4201BF2CEA020CD9
:1019B0001CF0803F50F8042B51F8043BF2D04FEA62
:1019C00002604FEA1222012828BFB0EB036F08BF64
:1019D0001B0AF4D003F0FF03000EC01A704710F08A
:1019E000030F0AD010F8012B11F8013B012A28BF80
:1019F0009A42F4D0A2EB030070474DF8045D50F812
:101A0000042B01F0030521F0030151F8043B022DE2
:101A100026D04DD822F07F45B5EB132FA2F1013C23
:101A20002CEA020C0DD11CF0803C08BF51F8043B9D
:101A30000AD185EA0205B5EB036F0CD150F8042BEF
:101A4000E8E74FEA13235BE03CF07F4C54D10B787E
:101A50004FEA126554E04FEA126503F0FF034FE0CE
:101A60004FEA0245A2F1013C4FEA15452CEA020C6F
:101A7000B5EB134F18D11CF0803C08BF51F8043B64
:101A800007D185EA0205B5EB034F09D150F8042BC5
:101A9000E6E75FEA0C4C2FD10B884FEA12452FE0A6
:101AA0004FEA03434FEA12454FEA134328E000BFD1
:101AB00002F0FF05B5EB136FA2F1013C2CEA020C1A
:101AC0000DD11CF0803C08BF51F8043B0AD185EAD7
:101AD0000205B5EB032F0AD150F8042BE8E74FEAD3
:101AE00013630DE012F0FF0F06D051F8043B4FEAEC
:101AF000122523F07F4303E04FF0000020BC704725
:101B000005F0FF0203F0FF00012828BF904204BF48
:101B10002D0A1B0AF4D0A2EB000020BC704700BFC6
:101B200020F0030110F00300C0F1000051F8043B65
:101B300000F1040C4FEACC0C6FF000021CBF22FA3B
:101B40000CF213434FF0010C4CEA0C2C4CEA0C4CF9
:101B5000A3EB0C0222EA030212EACC1204BF51F8F2
:101B6000043B0430F4D0C2F1000102EA0102B2FAEF
:101B700082F2C2F11F0200EBD20070472DE9F04F54
:101B8000D7B01C46914609910546189003F01CFCFD
:101B900002680D9410461A92FFF7C2FF19901DB10A
:101BA000AB6B002B00F04582099BB3F90C205B6EF8
:101BB00091B2DE0702D48D0540F1A286880409D4D3
:101BC000099B42F400529A8191B21A465B6E23F44B
:101BD000005353660A0740F1BC80099B1B69002B28
:101BE00000F0B78001F01A030A2B00F0C080002437
:101BF0002DAB224698464D46CDE92B442A931494AA
:101C000000230024CDE916342B78CDE91B22CDE941
:101C10001E22DDF860B01D920A92002B00F07D813B
:101C2000A94604E019F8013F002B00F0B580252BF0
:101C3000F8D1B9EB050640F0B38099F80030002BDD
:101C400000F06B8100234FF0FF3A2B21202499F8FC
:101C500001708DF88B3009F101090B93079309F19D
:101C60000109A7F120035A2B00F2CE80DFE813F020
:101C70004303CC00CC003C03CC00CC00CC001903C7
:101C8000CC00CC000C030703CC000003E702CC001F
:101C9000E0025B005B005B005B005B005B005B00E5
:101CA0005B005B00CC00CC00CC00CC00CC00CC00B6
:101CB000CC005C01CC001102E5015C015C015C011F
:101CC000CC00CC00CC00CC00CE02CC00CC00440236
:101CD000CC00CC00CC001F02CC00BA02CC00CC005F
:101CE0008C07CC00CC00CC00CC00CC00CC00CC00CD
:101CF000CC005C01CC001102E9015C015C015C01DB
:101D0000B002E9016A00CC00A602CC007B024802C6
:101D100093026A00CC001F026E008807CC00CC0042
:101D20006407CC006E000022A7F1300319F8017B94
:101D300002EB820203EB4202A7F13003092BF5D933
:101D40000B928EE7079B43F02003079399F80070EE
:101D500085E7099D1898294601F05CFD002841F0AF
:101D60004883A98901F01A030A2B7FF440AF099A2E
:101D7000B2F90E30002BFFF63AAF536EDE0702D4F5
:101D80008D0541F16F8123464A460999189857B04D
:101D9000BDE8F04F01F09ABCB9EB050600F0BD803C
:101DA0002C9BC8E9005633442C932B9B0133072B03
:101DB0002B9305DC08F108080A9B33440A933CE79F
:101DC000584609992AAA05F0BFF880B90DF1B40860
:101DD000F2E7584609992AAA05F0B6F8002800F05B
:101DE0008D800E9B1BB11946189803F02BF8099BA8
:101DF0005A6E9B89D40740F11381590601F105837E
:101E00000A9857B0BDE8F08F002F00F086800123BC
:101E100000228DF8F47008933DAD8DF88B200C9363
:101E200092460E92109215921392079B13F00203A2
:101E30000F9302D0089B02330893079B2C9C13F04E
:101E40008403129305D10B9B08995E1A002E00F3B0
:101E5000AF8082B10122C8F804202B9A01340132EC
:101E60000DF18B01072A2C942B92C8F8001000F377
:101E7000D38308F108080F9B7BB10223C8F8043014
:101E80002B9B0234013323AA072B2C942B93C8F8E5
:101E9000002000F3CD8308F10808129B802B00F08E
:101EA000B8820C9BAAEB0306002E00F3F582079B79
:101EB000DE0500F155820C9BC8F800501C44C8F8A0
:101EC00004302B9B2C940133072B2B9300F36C8352
:101ED00008F10808079B5D0705D50B9B089A9D1A1A
:101EE000002D00F3B183DDE90A3208998A42ACBFC4
:101EF0009B185B180A93002C7FF46BAF00232B9385
:101F00000E9B1BB158460E9902F09CFF4D460DF1F9
:101F1000B4082B78002B7FF483AE2C9B002B41F070
:101F2000548200232B9362E70D9B073323F00702B3
:101F3000F2E80234CDE9163424F000441E46184677
:101F40000D9221464FF0FF32B44B07F0D1F8002834
:101F500040F02285304621464FF0FF32AF4B07F06C
:101F6000A9F8002840F01885DDE9160100220023B9
:101F700007F096F8002840F08B879DF88B20002111
:101F80000320079BA64D23F080030793A54B0E91DA
:101F90000890472FC8BF1D468A460C901091159196
:101FA0001391002A3FF441AF089B013308933CE7AB
:101FB000102E2B9A23DD21461023099C04E0103EAD
:101FC000102E08F1080819DD013297481031072A50
:101FD000C8E90003CDE92B21F1DD214658462AAAA4
:101FE00004F0B2FF00287FF4FCAEDDE92B21103EA7
:101FF000102E4FF010030DF1B408E5DC0C46013251
:10200000894B3444072ACDE92B24C8F80460C8F86A
:10201000003000F387869DF88B2008F1080818E748
:1020200098053FF5EAAE099CA06D03F02DFAA3894F
:10203000E3E6189802F090FDB6E5079B43F0100325
:102040000793079B980640F13A840D9B073323F0D2
:1020500007031A465B6852F8084B1E460D92002B88
:10206000C0F23E84BAF1FF3F079B00F0C58223F027
:10207000800354EA0602089340F0BF82BAF1000FD1
:1020800040F0C08207934FF0000A56ADCDF830A063
:1020900059E1012000220D9B089053F8041B3DAD2F
:1020A000CDE90C038DF88B208DF8F410B8E60026EE
:1020B0000D9C8DF88B6054F8045B002D00F0BB85FF
:1020C000BAF1FF3F00F0858652463146284603F0BC
:1020D00071FD0E90002801F05B810E9BB2465B1BE8
:1020E000CDE90C3423EAE3739DF88B2008930E9618
:1020F00010961596139654E7079B43F01003079329
:10210000079B13F0200600F0B5830D9B073323F0E7
:1021100007035E6853F8084B0D93079B23F4806315
:102120000893002300228DF88B20BAF1FF3F00F0C6
:10213000EE80089A22F08002079254EA060240F0EC
:10214000E480BAF1000F40F03B82002B9BD1089B4A
:1021500013F001030C9300F0DC8330230DF25715CC
:102160008DF85731EFE00D9A52F8043B0D92079A23
:10217000910600F10A84079AD20600F10686079AB2
:10218000570600F1AF86079A960540F1FE850A9A38
:102190004D461A70BDE6079A782742F0020208926F
:1021A00030220D9B8DF88C2053F8044B1F4A0D9361
:1021B000002602238DF88D701B92B3E799F800700A
:1021C000079B6C2F00F02E8543F01003079346E524
:1021D00099F80070079B682F00F01B8543F04003BF
:1021E00007933CE5079B43F010030893089B13F00B
:1021F000200600F051830D9B073323F007031A4696
:1022000052F8084B5E680D9201238BE7079B99F803
:10221000007043F00803079321E500BFFFFFEF7F45
:1022200034C2000838C2000878C2000844C200085E
:10223000079B99F8007043F0800307930FE54A4627
:1022400012F8017B2A2F01F00A82A7F13003092B33
:1022500091464FF0000A3FF604AD19F8017B0AEBF6
:102260008A0A03EB4A0AA7F13003092BF5D9F8E4EF
:1022700099F80070079B43F004030793EFE499F883
:1022800000708DF88B10EAE40D9B99F8007053F8FC
:10229000042B002A0B920D93BFF6E1AC53420B9333
:1022A000E8E7584603F090F8436818461E93FFF796
:1022B00037FC034658461E461F9303F085F8836893
:1022C0002B211D93002E3FF441AD1D9B99F800700A
:1022D000002B3FF4C4AC1B78002B3FF4C0AC079B31
:1022E00043F480630793BAE4079B99F8007043F0C6
:1022F00001030793B3E49DF88B3099F80070002B2D
:102300007FF4ADAC8DF88B40A9E4079A0892012BBD
:1023100000F07381022B00F05B8156AD04F00703DF
:10232000E40844EA4674F608303354EA06012A46C3
:1023300005F8013DF2D10899C80700F1538256AB68
:102340005B1B07910C930C9A00235245B8BF524671
:102350000E93089210939DF88B201593139320E60B
:10236000652F40F3D380DDE916010022002306F03B
:102370008DFE002800F0A5810123C8F804302B9BB6
:10238000B44A01330134072B2C942B93C8F8002056
:1023900000F3E18408F10808249B149A934280F228
:1023A000AA82199B1A9A1C44C8E900232B9B2C94DF
:1023B0000133072B2B9300F31F8408F10808149BAB
:1023C0005D1E002D7FF786AD102D2B9A41F34481C1
:1023D000A14B10261F46DDF824A005E008F10808EF
:1023E000103D102D40F3C48401321034072AC8E98F
:1023F0000076CDE92B24F1DD514658462AAA04F097
:10240000A3FD00287FF4EDACDDE92B240DF1B40829
:10241000E6E70B9B089A9E1A002E7FF742AD102E1E
:102420002B9A8D4B25DD21461C464346A846099D27
:1024300004E0103E102E03F1080316DD10200132D7
:102440001031072ACDE92B211C605860F1DD2946A7
:1024500058462AAA04F078FD00287FF4C2ACDDE9D2
:102460002B21103E102E2DABE8DC45469846234626
:102470000C4601323444072ACDE92B24C8F8003039
:10248000C8F8046000F3A3830C9B08F10808AAEBCA
:102490000306002E7FF70BAD102E2B9A40F3F58428
:1024A0006D4B21464FF0100A1C464346A846099D35
:1024B00004E0103E102E03F1080315DD0132103147
:1024C000072AC3E9004ACDE92B21F2DD2946584607
:1024D0002AAA04F039FD00287FF483ACDDE92B2122
:1024E000103E102E2DABE9DC4546984623460C469F
:1024F00001323444072ACDE92B24C8F80030C8F84B
:10250000046000F3AA8108F10808D0E4149A2B9B18
:10251000012A04F1010408F1080603F1010740F360
:102520004E810123072FCDE92B74C8F80050C8F85D
:10253000043000F39D83199B01371A9A1C44072F1E
:10254000C6E90023CDE92B7400F39E830836149A64
:102550007B1C0F930C9302F1FF3A0023DDE9160177
:10256000002206F1080806F091FD002840F048819D
:102570000C9B01355444072B3560C6F804A02C94FD
:102580002B9300F3148306F1100346469846BA1CB9
:102590000C921C9B0C9A1C447360072A26AB2C944B
:1025A0002B9233607FF796AC584609992AAA04F01B
:1025B000CBFC00287FF415AC2C9C0DF1B40889E409
:1025C000012B00F05087022B079B08937FF4A5AEE8
:1025D0001B9A56AD04F00F03D35C240944EA067439
:1025E000360905F8013D54EA0603F3D1089B079329
:1025F00056AB5B1B0C93A6E608930A2C76F10003FE
:1026000080F04E83089B3034079301238DF85741A7
:102610000C930DF2571596E6584609992AAA04F02C
:1026200093FC00287FF4DDAB2C9C0DF1B40822E470
:10263000584609992AAA04F087FC00287FF4D1ABF8
:102640002C9C0DF1B40828E4102D2B9B23DD1026C3
:10265000099F08E074C2000888C20008103D102DD0
:1026600008F1080817DD0133AB4A1034072BC8E91D
:102670000026CDE92B34F1DD394658462AAA04F06C
:1026800063FC00287FF4ADABDDE92B34103D102D49
:102690000DF1B408E7DC01339F4A2C44072BCDE948
:1026A0002B34C8F80450C8F800207FF71CAC5846FB
:1026B00009992AAA04F048FC00287FF492AB2C9CCC
:1026C00011E4249B002B40F32B81DDE913739F421F
:1026D000A8BF1F46002F0BDD2B9B3C440133072B6B
:1026E000C8E900572C942B9300F3DE8508F1080805
:1026F000139E002FA8BFF61B002E00F37B83079BC1
:10270000DDF84CA05805AA4400F1DF84249B149AFC
:10271000934203DB079AD10740F1DB83199A1A9998
:102720001444C8E900122B9A2C940132072A2B92E8
:1027300000F3C78508F10808149AAE18A6EB0A063C
:10274000D51AAE42A8BF2E46002E0DDD2B9B344479
:102750000133072BC8F800A0C8F804602C942B9311
:1027600000F3238608F10808002EA8BFAD1B002D3A
:102770007FF7B0AB102D2B9A40F36E87674B102676
:102780001F46DDF824A005E008F10808103D102DD3
:1027900040F3EE8201321034072AC8E90076CDE911
:1027A0002B24F1DD514658462AAA04F0CDFB00281F
:1027B0007FF417ABDDE92B240DF1B408E6E7079AA7
:1027C000D2073FF5AEAE0122072FCDE92B74C8F832
:1027D0000050C8F8042000F3268502330C9308F15A
:1027E0001008D6E6302B3FF401AF089B023A07935E
:1027F000302305F8013C56AB9B1A15460C93A2E515
:10280000BAF1000F7FF7C5AEBAF1100F40F312878F
:10281000424B10251A46DDF8248023460F9F1446AC
:1028200006E0AAF1100ABAF1100F40F3B0810137A7
:102830001033072FC6E900452C9306F108062B97A5
:10284000EFDD414658462AAA04F07EFB00287FF4BB
:10285000C8AADDE92B732DAEE3E7584609992AAAE9
:1028600004F072FB00287FF4BCAA2C9C0DF1B40884
:10287000FFF71DBB079A0D9912F0100201F1040336
:1028800040F05681079911F0400100F0DA820D996D
:1028900016460C880D9340E4089A0D9912F0100228
:1028A00001F1040340F03F81089911F0400100F06C
:1028B000DD820D9916460D930C88012332E40799A9
:1028C0000D9AC90602F1040359D4079A520650D54D
:1028D0000D9A0D93B2F90040E6173346FFF7BFBBE0
:1028E000079B644208934FF02D0366EB46068DF874
:1028F0008B30012319E4079BDD077FF5EBAA50E538
:10290000099DA86D02F0B8FDB5F90C2091B2FFF752
:1029100055B956AD17E500BF78C2000888C2000857
:102920000122C8F804202B9AAF4901320134072A4A
:102930002C942B92C8F8001000F39B8408F108082F
:10294000002B40F02782079B149A03F001031343E6
:102950003FF4C0AA199B1A9A1C44C8E900232B9A79
:102960002C940132072A2B9200F36E8308F1080899
:1029700021E2079A12F4007F0D9A40F0B8821468A1
:102980000D93E6173346FFF76ABB0A9A4D461A6065
:10299000D2175A60FFF7BDBADDE9160102460B46B1
:1029A00006F0A6FB002840F0E385612F00F0988533
:1029B000412F00F0A78227F02003BAF1FF3F0893D0
:1029C00000F0BB85472B04D1BAF1000F08BF4FF0D0
:1029D000010ADDE91601079C0E1E44F48073C0F263
:1029E0003B84079300230F9412930C900E93089B43
:1029F000462B00F07484452B0C9A00F03885022198
:102A0000009128A9049125A9039124A93346584689
:102A1000CDF804A0029100F0FFFF089B0546472B6C
:102A200040F032860F9BDB0700F11A85289B5B1B69
:102A30001493249B1393089B472B00F01883089B47
:102A4000462B00F07A840899139BFAB2412908BFFB
:102A50000F3203F1FF3306BFD2B201210021002B58
:102A60008DF89820B4BF2D222B222493B8BF139B3E
:102A70008DF89920B8BFC3F10103092B40F3AD8550
:102A80000DF1A70C6246594E1C46104686FB0312F8
:102A9000D917C1EBA20101EB8102A3EB4202303254
:102AA000632C00F8012C0B4600F1FF32ECDC3033D4
:102AB000811EDBB28C4502F8013C40F2E1850DF14C
:102AC0009A0101E012F8013B944501F8013BF9D16C
:102AD0000DF1A9030DF19A021B1A134426AA9B1AA1
:102AE0001C93149B1C9A012B1A440C9240F3908562
:102AF0000C9B199A13440C930F9B0C9A23F480633C
:102B000043F480730793002322EAE2721093089241
:102B100015931393129B002B40F0D0829A469DF898
:102B20008B20FFF73EBA0D930C680123FFF7FABA2A
:102B30000C680D93FFF7F1BA2D4B1B93079B13F015
:102B4000200600F08B800D9B073323F007035E689F
:102B500053F8084B0D93079BDD070AD554EA06028C
:102B600007D043F00203079330238DF88D708DF862
:102B70008C30079B23F4806308930223FFF7D2BABB
:102B8000079B0893FFF732BB1A4B1B93D6E72246ED
:102B90001C4613467A1C0C9206F10808C6E9003A56
:102BA0000C9B5444072B2C942B9340F38B81584659
:102BB00009992AAA04F0C8F900287FF412A92B9BCE
:102BC0002C9C01330C932DAE0DF1BC08E1E458466A
:102BD00009992AAA04F0B8F900287FF402A92C9CCC
:102BE0000DF1B408FFF75DB974C200086766666648
:102BF00044C2000858C20008584609992AAA04F09D
:102C0000A3F900287FF4EDA82C9C0DF1B408FFF780
:102C1000D6BB43F4007399F80170079309F10109D9
:102C2000FFF71DB843F0200399F80170079309F1ED
:102C30000109FFF714B85346062BAA4628BF0623FE
:102C40002A460E950893AD4D0D940C93CDF840A0F7
:102C5000CDF854A0CDF84CA0FFF7A3B9079A0D9971
:102C600012F0100201F104036BD00C680D9372E7AF
:102C7000584609992AAA04F067F900287FF4B1A8F8
:102C8000DDE92B742DAE56E4584609992AAA04F0C2
:102C90005BF900287FF4A5A8DDE92B742DAE56E47E
:102CA0000023089956AA01F48061CDE90EA8079780
:102CB000CDF83090174699468A46DDF874800CE0CE
:102CC0000023204631460A2206F050FA0A2C76F1FB
:102CD00000031DD304460E462F4620460A22002339
:102CE000314606F043FA30327D1E09F1010907F83A
:102CF000012CBAF1000FE3D098F800309945DFD1EC
:102D0000B9F1FF0FDCD00A2C76F1000380F0C5800A
:102D1000CDF87480CDF85090079FDDF83090DDE954
:102D20000EA863E4584609992AAA04F00DF9002870
:102D30007FF457A89DF88B202C9C0DF1B408FFF769
:102D400088B8079911F0400100F086800D99164669
:102D50000C880D93FFE6584609992AAA04F0F4F866
:102D600000287FF43EA82C9C0DF1B408FFF714BB9B
:102D70003B4601322C44072AC8F80030C8F80450FA
:102D8000CDE92B247FF7A4A80EE40A9A4D461A60D9
:102D9000FFF7BFB8199A1A991444C8E900122B9A80
:102DA0002C940132072A2B9200F34E8108F1080877
:102DB000002BC0F22F83149B01321C44072ACDE95B
:102DC0002B24C8F80050C8F804307FF781A8FFF71B
:102DD000EBBB28460D94FEF7A3FE20EAE073B24653
:102DE0009DF88B200C900E961096159613960893CE
:102DF000FFF7D7B8102E2B9A40F33C84404B102796
:102E00001946DDF824A023460C4605E008F1080821
:102E1000103E102E40F3F58101321033072AC8E925
:102E20000047CDE92B23F1DD514658462AAA04F08C
:102E30008BF800287EF4D5AFDDE92B230DF1B40823
:102E4000E6E7079A12F400760D9A1ABF0E46147838
:102E500014680D93FFF761B9079A12F400760D9A82
:102E60001ABF0E46147814680D9374E6089A12F48B
:102E700000760D9A18BF0E460D9318BF14784FF0C8
:102E8000010308BF1468FFF74DB91D4BFFF730BBB6
:102E90002D228DF88B20FFF772B81F9B1E99ED1A1B
:102EA0001A46284603F0E0FF98F801300BB108F10C
:102EB0000108204631460A2200234FF0000906F09F
:102EC00055F907E7013346460C9308F10808FFF768
:102ED00060BB149AAE18A6EB0A06D51AAE42A8BF7C
:102EE0002E4641E40A9A4D461A80FFF712B892F92D
:102EF00000400D93E6173346FFF7B1B86CC20008E7
:102F000088C2000830238DF88C3058238DF88D301E
:102F1000079BBAF1630F43F002030F9300F3D582CE
:102F200000233DAD0E93079B43F48173079327F075
:102F300020030893179B1E1EC0F29381169B0C93CF
:102F400000231293612F00F03083412F7FF44FADA7
:102F500024AA31460C9803F005FF00224FF07F535E
:102F600005F02CFE02460B46CDE91023002200237B
:102F700006F08CF808B101232493B34B0C93CDE9F0
:102F80001379CDF880802C46DDE910890AF1FF36EF
:102F9000CDF840B0CDF854A0DDF830B0219505E073
:102FA00000220023013E06F071F8E0B90022A74B91
:102FB0004046494605F002FE8946804606F0AEF8D6
:102FC000054605F091FD0B4602464946404605F090
:102FD0003DFC1BF80530A24604F8013B731C374644
:102FE00080468946DCD1404649460022984B3E4601
:102FF000DDF85090139FDDF840B0CDF84CA014954B
:10300000CDE91001DDF854A0DDF88080219D06F0A7
:1030100065F8002840F03D82DDE9100100228C4B6C
:1030200006F034F818B1149BD90700F13282002E53
:10303000334606DB30220133234404F8012BA3423C
:10304000FBD1631B1493F4E4584609992AAA03F0B0
:103050007BFF00287EF4C5AEDDE92B24249B0DF117
:10306000B408A5E6906D02F00FFAFEF78CBE139B34
:10307000DA1C01DB534504DD023F27F020030893EF
:10308000E1E4DDE913329A4200F3A9810F9AD407F3
:1030900040F18682199A13440C930F9B580540F116
:1030A0008282139B6727002B00F35A810C9B23EA33
:1030B000E37308930023109315932BE52D224FF013
:1030C000000A8DF88B20FEF76FBF149B4246DDF897
:1030D0005480EB1856460C93CDF83C9021461D9F2A
:1030E000DDF87C90DDF824A0109B1295B8F1000F5C
:1030F0002ED0002B6AD1013F08F1FF381E9B4944B6
:10310000C2E900392B9B2C910133072B2B9361DCF7
:1031100008320C9B38789B1B8342A8BF0346002BC8
:103120001C460ADD2B98194401300728C2E90063C8
:103130002C912B9059DC38780832002CB4BF05460E
:10314000051B002D14DC0644109BB8F1000FD0D1F4
:10315000002B3BD1129D149BB246EB189E42904629
:103160000C4628BF9A46DDF83C901D97FFF7CEBA73
:10317000102D2B981DDD102404E0103D102D02F1C0
:10318000080216DD0130334B10310728C2E9003444
:10319000CDE92B01F1DD514658462AAA03F0D4FEB1
:1031A00000287EF41EAEDDE92B01103D102D2DAA66
:1031B000E8DC0130274B29440728CDE92B01556075
:1031C000136064DC387808320644BDE7109B013B8D
:1031D000109393E7514658462AAA03F0B5FE0028FB
:1031E0007EF4FFAD2C992DAA93E7514658462AAAA2
:1031F00003F0AAFE00287EF4F4AD38782C992DAAAD
:103200009BE721461C460B4601323444072ACDE990
:103210002B24C8F80030C8F8046000F3668108F178
:103220000808FFF76CBA584609992AAA03F08CFEE1
:1032300000287EF4D6AD2B9B2C9C01332DAE0C9335
:103240000DF1BC08FFF7A5B958C2000800003040D6
:103250000000E03F88C20008079A079300230F92FE
:103260000E932D22DDE9163412920C9304F10046E0
:1032700068E6584609992AAA03F066FE00287EF4FB
:10328000B0AD249B2C9C0DF1B408FFF759BB5146FF
:1032900058462AAA03F058FE00287EF4A2AD3878DA
:1032A0002C992DAA06444FE7584609992AAA03F0FB
:1032B0004BFE00287EF495AD2C9C0DF1B408FFF771
:1032C00017BA584609992AAA03F03EFE00287EF450
:1032D00088AD249B2C9C0DF1B408FFF72DBA032177
:1032E000009128A9049125A9039124A933465846A1
:1032F0000C9ACDF804A0029100F08EFB03780546ED
:10330000302B00F07881249B5344EC183146002286
:1033100000230C9805F0BAFE10B12346FFF787BBD7
:10332000289BA342BFF483AB30215A1C289219700A
:10333000289B9C42F9D8FFF77ABB0F9B139A03F0A6
:103340000103002A43EA0A0340F37781002B40F08F
:10335000F8806627139B0C930F9B5A057FF5A6AE4A
:103360001D990B78FF2B00F087810024139A2046CB
:1033700004E001300131FF2B00F0E980934280F23C
:10338000E680D21A4B78002BF3D10B780134F2E7A8
:10339000CDF820A0CDF830A09DF88B2082460D946A
:1033A000109015901390FEF7FCBD584609992AAA73
:1033B00003F0CAFD00287EF414AD249D149B2C9CC0
:1033C0000DF1B4085D1BFFF7CFB9099918982AAA27
:1033D00003F0BAFD00283EF4A4ADFEF708BD149B2F
:1033E000199A9A18139B0C92002B40F317816727A8
:1033F000B2E7099B5B6EDB0707D4099B9B899F059E
:1034000003D4099B986D02F03FF84FF0FF330A9305
:10341000FEF7F6BC5E42103380F24081A04B1027CD
:103420001946DDF824A023460C4604E008F10808FC
:10343000103E102E66DD01321033072AC8E900471E
:10344000CDE92B23F2DD514658462AAA03F07CFD34
:1034500000287EF4C6ACDDE92B230DF1B408E7E7C4
:1034600005EB0A0452E7079B0893FFF7CBB802214C
:10347000009128A9049125A90AF10104039124A926
:10348000019433465846029100F0C6FA05462C4492
:103490003CE7139B28930C9B14F8012CD97B234603
:1034A0008A4209D1302003F8010C289B5A1E289229
:1034B00013F8012C9142F6D0392A0BBF0C9A013235
:1034C000927AD2B203F8012CBBE558460AF1010109
:1034D00002F08CF80546002800F0D9800E9022E515
:1034E00030238DF88C30782310E5584609992AAAA4
:1034F00003F02AFD00287EF474AC2C9C0DF1B40876
:10350000FFF7FDB821461C460B4601323444072A1A
:10351000CDE92B24C8F80030C8F804607FF726AA4C
:10352000584609992AAA03F00FFD00287EF459ACE9
:10353000DDE92B240DF1B4083DE44FF0060AFFF756
:1035400048BA199B6627D31853440C9304E71D917E
:10355000139215901094109A159B1F9913440C9A6E
:1035600001FB03230C9323EAE3730893FFF7D2BA1A
:10357000179B0320002B079BB8BF2D2223F080034D
:1035800007934FF00003A8BF9DF88B2019460E93B8
:10359000444D454BB8BF8DF88B200890FEF7F9BC21
:1035A000139B0C9379E5672780E524AA31460C9894
:1035B00003F0D8FB00224FF07F5305F0FFFA0246DC
:1035C0000B46CDE910230022002305F05FFD08B172
:1035D00001232493354B0C93D1E441BB30228DF869
:1035E0009A200DF19B02303302F8013B26ABD31A2F
:1035F0001C93FFF776BA3146002200230C9805F0A1
:1036000045FD00287FF47FAECAF1010324937BE6D9
:103610000F9BDE077FF570AAFFF76ABAC3F10103BB
:103620001A4422EAE27367270C92089342E50DF1EF
:103630009A02D8E71A4BFFF7B1BA23B901236627DC
:1036400008930C9336E5199B6627013353440C937A
:1036500023EAE37308932DE5114BFFF78ABB0D9B1B
:1036600099F80170914653F8042B0D9342EAE27ADF
:10367000FEF7F5BA0A4BC7E50023109315936AE7E6
:1036800002231C93FFF72DBA54462C443EE6099AB8
:10369000938943F040039381FEF7A9BB004B34E7C5
:1036A00088C200083CC2000840C2000844C20008AA
:1036B0008C4600B586461346034A714610685DF88D
:1036C00004EB6246FEF75ABA14000020F0B54FF43E
:1036D000806C1546002406461F46ADF26C4D1AABB1
:1036E000009304938B8916A823F00203ADF80C30E5
:1036F0004B6E06941993CB890C46ADF80E30CB690E
:10370000CDF808C007934B6ACDF814C0099301F0B7
:10371000ABFE2A463B4669463046FEF72FFA051EA9
:1037200007DB6946304601F06BF9002818BF4FF0FF
:10373000FF35BDF80C305B0603D5A38943F0400389
:10374000A381169801F094FE28460DF26C4DF0BD51
:10375000F8B506460D46144610B1836B002B43D0D6
:10376000B4F90C20A3691007A36091B21BD523699B
:10377000CBB1EDB289042F4622D522686169D31AF4
:10378000994229DD0133A1680139A160511C2160F2
:10379000157062699A422AD0A389DB0701D50A2DE8
:1037A00025D03846F8BD2146304600F033F820BB1E
:1037B000B4F90C20EDB291B289042F462369DCD410
:1037C00042F40052A281626E616922F40052626684
:1037D0002268D31A9942D5DC2146304601F010F90F
:1037E00058B901232268CEE701F0B6F9B8E72146BF
:1037F000304601F005F90028D3D04FF0FF37D0E76D
:1038000003460A46024908681946FFF7A1BF00BFF0
:103810001400002038B5334B05461B680C460BB12D
:103820009A6B12B3B4F90C3018079AB225D52169F6
:1038300000292DD012F0010007D000256069A56095
:103840004042A06139B1002038BD950758BF60697A
:10385000A0600029F7D1120658BF0846F4D543F0FE
:1038600040034FF0FF30A38138BD184601F074F9D2
:10387000B4F90C3018079AB2D9D4D1062AD5520718
:1038800014D4216943F00803A3819AB20029D1D14D
:1038900002F42070B0F5007FCCD02146284601F01C
:1038A000F5FDB4F90C3021699AB2C3E7216B51B12F
:1038B00004F14002914204D0284601F0C3FAB4F961
:1038C0000C30002222630022216923F02403C4E982
:1038D0000012D7E7092243F040032A604FF0FF307F
:1038E000A38138BD140000202DE9F04F03690C6955
:1038F00085B0A342C0F28980013C01F11405A30008
:1039000000F11408019355F8243058F824200133AD
:103910008A469A4208EB84018146B2FBF3F605EB36
:10392000840702913AD30021AE4640460A46A34698
:1039300003955EF8045B0468ABB206FB03132D0C21
:10394000190C06FB05119BB2D21A1FFA84FC944491
:103950008AB2C2EB144202EB2C421FFA8CFC4CEAF6
:103960000243774540F8043B4FEA11414FEA2242B7
:10397000DFD2019B5C4658F80330039D73B9029B6C
:10398000043B984504D307E0984504F1FF3403D283
:1039900053F80429002AF7D0C9F810405146484688
:1039A00002F076FD00282CDB40460023013655F856
:1039B000041BD0F800C08AB29A1A1FFA8CFE0B0CB6
:1039C0007244C3EB1C4303EB224392B242EA03422C
:1039D000AF4240F8042B4FEA2343E8D258F82420A2
:1039E00008EB84036AB9043B984504D307E0984583
:1039F00004F1FF3403D253F80429002AF7D0C9F8A0
:103A00001040304605B0BDE8F08F002005B0BDE89D
:103A1000F08F00BF000000002DE9F04F16461F4652
:103A2000016C9BB00446CDE90267279D41B101239B
:103A3000426C93408B604A6002F07AFA0023236460
:103A4000B7F10009B4BF012300232B60784BBCBF42
:103A500029F00049CDF80C9033EA090300F0AD805D
:103A6000DDE902231046194600220023CDE90801B2
:103A700005F00CFB804670B10123269A1360289B49
:103A8000002B00F0E9826B481860431E04930498F1
:103A90001BB0BDE8F08F18AB019319AB0093204623
:103AA000DDE9082302F03EFE5FEA1955834640F047
:103AB0009A80DDE91885454405F23243202B40F316
:103AC000B383C3F1400305F2124009FA03F926FA61
:103AD00000F049EA000004F0F7FF0123013D0E93D6
:103AE000A1F1F8710022544B04F0B0FE4AA3D3E9CF
:103AF000002305F063F84AA3D3E9002304F0A8FEED
:103B0000064628460F4604F0EFFF47A3D3E90023FB
:103B100005F054F802460B463046394604F098FE4C
:103B200006460F4605F0FAFA002282460023304688
:103B3000394605F0B5FA002840F08182A8EB05056A
:103B40006B1EBAF1160F059300F26D82DDE90801D4
:103B50003A4B03EBCA03D3E9002305F0A1FA00288E
:103B600072D000230D936B1E002B0AF1FF3AC0F2B6
:103B7000608200230A93BAF1000F6BDA0A9BCDF83A
:103B800018A0A3EB0A030A93CAF100030C93249B29
:103B90004FF0000A092B66D8052B40F3438300251C
:103BA000043B2493249B023B032B00F25D86DFE859
:103BB00013F05B0458044F04320442F20F73269A48
:103BC000C9F31309136059EA06031CD1289B002B83
:103BD00000F059861A4B04930833289A049813600E
:103BE0001BB0BDE8F08FDDE90812C2F313030846ED
:103BF00043F07F51CDF83880A5F2FF35DDF86080C5
:103C000041F440116EE7289B002B40F0E7830D4BF9
:103C100004933CE7AFF3008061436F63A787D23F13
:103C2000B3C8608B288AC63FFB799F501344D33FAB
:103C30000000F07F75C200080000F83F78C300085C
:103C40009CC2000898C200086B1E002BC0F27C8446
:103C50000D900A90059B5344CDE9053A00230C933F
:103C6000249B092B98D9002324934FF0FF3301257F
:103C7000079300230B9525930021079B61640F9305
:103C8000204602F02FF90490002800F0F585049BEF
:103C90002364079B0E2B00F21481002D00F011818C
:103CA0000699002940F35284AF4B01F00F0203EB59
:103CB000C203C8054FEA2115D3E9006740F1088423
:103CC000DDE90801A94B4FF00309D3E9082305F00A
:103CD0009FF8CDE9100105F00F058DB1DFF88C825A
:103CE000E90709D5D8E900233046394604F066FFD4
:103CF00006460F4609F101096D1008F10808EFD1D9
:103D0000DDE910013B46324605F082F80746884659
:103D10000D9B43B1002238464146954B05F0C0F952
:103D2000002840F02985484604F0DEFE3A46434626
:103D300004F044FF8F4B002204F08AFD079B0546E8
:103D4000A1F15076002B00F0A080069B1693079BF4
:103D50001093049B41463846CDE912565E1C05F08F
:103D6000DDF91099804B00F1300503EBC10353E9F5
:103D70000212CDE9141204F0B7FE02460B46384693
:103D8000414604F063FDDDE9142389460B99804622
:103D9000EDB2002900F098840020774905F038F84A
:103DA000DDE9122304F052FD02460B46049FCDE9E3
:103DB00012233D7042464B4605F090F9002840F032
:103DC000CD84109DCDF85CA0CDF850B00027DDE982
:103DD00012AB10942AE00137AF4280F213855046AF
:103DE00059460022654B04F0E9FE0022634B8246EF
:103DF0008B464046494604F0E1FE8946804605F080
:103E00008DF9044604F070FE02460B4640464946D2
:103E100004F01CFD303452465B4606F8014B8046E8
:103E2000894605F03DF9002840F0E58442464B46BE
:103E300000204F4904F00AFD52465B4605F030F978
:103E40000028C8D03546DDF850B0109C169B049A67
:103E50000133069302E0954200F0B4842E4615F833
:103E6000013D392BF7D00133DBB22B70BFE148465F
:103E700004F03AFE3A46434604F0A0FE00223D4BD1
:103E800004F0E6FC0546A1F15076414600223C4B89
:103E9000384604F0DBFC804689462A463346CDE9A5
:103EA000108905F01BF98046002840F09784DDE971
:103EB00010012A4606F1004305F0F2F8002840F010
:103EC0003A83199B002BC0F28F80069A0E2A00F3CA
:103ED0008B80254B03EBC203D3E9009A259B002B73
:103EE0001ADA079B002B17DC40F023830022244BB7
:103EF0004846514604F062FE02460B46DDE90801E1
:103F000005F0D8F8DDF81C804546002800F0C38293
:103F1000259B049EDB43C4E24A46DDE9086753461D
:103F20003046394604F074FF05F0F8F8804604F096
:103F3000DBFD4A46534604F041FE049D0B46024613
:103F40003946304604F082FC08F1300305F8013BA5
:103F5000079B012B00F0588305944FF001081C4685
:103F6000CDF808B02CE000BF78C3000850C30008AB
:103F70000000F03F00001C400000E03F0000244033
:103F8000000014404A4653463046394604F040FF8C
:103F900005F0C4F8834604F0A7FD4A46534604F0F2
:103FA0000DFE08F101080B4602463946304604F082
:103FB0004DFC0BF13003A04505F8013B00F02083D8
:103FC0000022A74B04F0FAFD0022002306460F460C
:103FD00005F05CF80028D5D0069B2E460133DDF8AD
:103FE00008B0059C069302E10B9A002A3AD0249A65
:103FF000012A40F38F82079B5F1E0C9BBB42C0F2DD
:104000006182DF1B079B002BC0F23783059A1A449D
:1040100005920A9A16461A440A920121204602F095
:1040200089F8054621E001230D936B1E002BBFF696
:10403000A0ADC5F101030A93002305939BE550460B
:1040400004F052FD32463B4605F020F800287FF48C
:1040500075AD0AF1FF3A71E5824B049304981BB0E9
:10406000BDE8F08F0C9FDDE90A65002E0CDD059997
:1040700000290B4608DDB142A8BF33460A9AF61A5A
:10408000D21ACB1A0A9205930C9BD3B10B9B002B2F
:1040900000F05382002F10DD29463A46204602F0F8
:1040A00025F905465A462946204602F071F8804611
:1040B0005946204601F03CFFC3460C9BDA1B40F0FA
:1040C000D6820121204602F035F8BAF1000F804671
:1040D00000F3AF80249B012B40F385814FF0000952
:1040E0000120BAF1000F40F0B080059A104410F0A2
:1040F0001F0000F08E80C0F12003042B40F3C78323
:104100000A9BC0F11C00034402440A930644059232
:104110000A9B002B05DD59461A46204602F042F95B
:104120008346059B002B05DD41461A46204602F0DA
:1041300039F980460D9B002B40F03681079B002B00
:1041400040F31C810B9B002B40F09B80069B0133AE
:1041500006930126049FDDF81C9007E059460023D2
:104160000A22204601F0EEFE8346013641465846BB
:10417000FFF7BAFB4E4500F1300A07F801ABEDDB63
:10418000079B4FF00009002BCCBF1E460126049B65
:104190001E4459460122204602F004F94146834656
:1041A00002F076F9002816F8012C40F39E8104995C
:1041B000731E04E0994200F0A68113F8012D392AFC
:1041C00003F10106F6D001321A704146204601F093
:1041D000AFFE65B1B9F1000F05D0A94503D049463E
:1041E000204601F0A5FE2946204601F0A1FE5946D1
:1041F000204601F09DFE0023069A3370269B1A602C
:10420000289B002B3FF443AC04981E601BB0BDE814
:10421000F08F1C200A9B064403440A93059B034429
:10422000059375E70125BDE4C3F1200306FA03F009
:1042300051E401465246204602F058F8249B80463D
:10424000012B40F3AF814FF00009D8F8103008EB94
:104250008303186901F022FFC0F1200045E700BF89
:104260000000244074C20008294600230A22204688
:1042700001F068FE0F9B0546002B40F3E282CDE97A
:104280000673002E00F31781B9F1000F40F0D881BA
:104290002F46029B079903F00102049B0B921E46D6
:1042A000013B1944249B0791134308934146584608
:1042B000FFF71AFB0346294658469A460A9302F02E
:1042C000E7F83A4681464146204602F001F9C268C5
:1042D0000AF130038246002A42D10146584605932E
:1042E00002F0D6F8024651462046029201F020FE26
:1042F000029A059B1AB90899002900F08A82B9F13F
:10430000000F06F1010AC0F25981249949EA010916
:104310000B9951EA090100F05181002A00F3B181A3
:10432000079A3370B24200F0C781594600230A222F
:10433000204601F007FEBD42834629464FF00003A8
:104340004FF00A02204613D001F0FCFD3946054625
:1043500000230A22204601F0F5FD56460746A5E750
:1043600001462046029301F0E3FD0122029BC6E7CD
:1043700001F0E8FD56460546074697E7249B022BC9
:1043800078DC0B9B002B7FF47CAF069B414601330E
:1043900058460693FFF7A8FA049E00F1300A4FF042
:1043A000000906F801ABF4E64146584602F070F801
:1043B0000028BFF6C3AE594600230A22204601F06A
:1043C000C1FD069B83465F1E0B9B002B7FF44CAF09
:1043D0000F9B002B40F32D820793BAE6B24B049358
:1043E0000333FFF7FABBDDE9021200297FF476AE52
:1043F000C2F31303002B7FF471AEAC4B1340002BC0
:1044000000F0F0810A9B4FF0010901330A93059BEC
:104410000133059364E601230B93259B069A13440D
:104420000F930133012B1E46B8BF012607930021CD
:10443000172E61647FF724AC012204235B0003F193
:104440001400B042114602F10102F7D9616417E489
:1044500001230B93259B002B42DD1E460F930793F0
:10446000E5E700230B93D8E700230B93F2E70F9BBC
:1044700006970793079B002B7FF44AAD4146052220
:10448000204601F05FFD80465846414602F000F8A4
:1044900000287FF73DAD3122069B049E013306F8CC
:1044A000012B013341462046069301F041FD002DCA
:1044B0007FF499AE9BE629463246204601F072FF12
:1044C0000546E1E60C9B0C97FB1A9A44002799E5F8
:1044D000DDE908234FF00209CDE91023FFF7FDBB0A
:1044E000012325930793FFF7C7BB03D11AF0010FF0
:1044F0007FF45DAE731E01E013F8012D302A03F145
:104500000106F9D061E6069B049A01330693312334
:1045100013705AE60E9A002A00F0248103F2334306
:10452000059A0C9F1A4405920A9A16461A440A9252
:1045300073E54FF000084546EAE4594620460C9AD8
:1045400001F0D4FE8346BCE50D9072E500F00E81CB
:10455000DDE90801069A564B554205F00F0203EBC0
:10456000C203D3E9002304F029FB2D110746884636
:1045700000F06F8100234FF002094E4EEA0706D586
:10458000D6E9002304F01AFB012309F101096D109B
:1045900006F10806F2D1002B3FF4BAAB0746884675
:1045A000FFF7B6BB029B002B7FF44DAEDDE9021294
:1045B000C2F31303002B3FF420AF44E602965646A5
:1045C0009A46069B002A03F10103069312DD594621
:1045D0000122204601F0E6FE4146834601F058FFE5
:1045E000002840F30181BAF1390F00F0F1800A9BF5
:1045F00003F1310A029BA94683F800A03D46E4E599
:10460000D846059CDDF808B0069B024601330693A8
:104610000B4604F01DF94A46534606460F4604F081
:104620005DFD48B94A4653463046394604F02EFDF2
:1046300020B15FEAC87001D5049A0FE42E46D6E592
:104640002046696801F04EFC0646002800F005810E
:104650002B6905F10C0102339A000C3001F0F2FADB
:1046600031460122204601F09DFE074611E65946DB
:10467000204601F03BFE834623E50A9B079A9E1ADB
:10468000CBE4029656469A46069BBAF1390F03F1DF
:104690000103069300F09C80029A0AF10103A946E7
:1046A00013703D4691E500BF98C200080000F07FFE
:1046B00078C3000850C3000856469A46069BA94690
:1046C00001333D46069364E5DDE9120104F076FA14
:1046D000049BCDE912011D70109B012B00F0AF80EF
:1046E000109D049B1D440022714B4046494604F036
:1046F00065FA8946804604F011FD074604F0F4F996
:1047000002460B464046494604F0A0F8303706F80A
:10471000017BB54280468946E5D1DDE912010022E0
:10472000644B04F095F842464B4604F0B9FC00286F
:104730007FF48CABDDE9122300205E4904F086F89B
:1047400042464B4604F0CAFC00283FF4BAAB15F8C9
:10475000013C2E46302B05F1FF35F8D0169B013376
:10476000069344E5189BC3F13603D9E64FF00209DE
:10477000DDE90878FFF7CCBA079B002B3FF477AB55
:104780000F9B002B7FF79DAB1093069B3846013B98
:10479000414600221693464B04F010FA0246884622
:1047A000174609F1010004F09FF93A46434604F028
:1047B00005FA0022404B04F04BF80546A1F1507673
:1047C000FFF7C7BA069B0133069331232B700EE522
:1047D0003922029BA9461A703D46E8E44FF00008D2
:1047E000454658E699467BE47FF404AF1AF0010F82
:1047F0007FF4F9AEFEE6169BDDF850B00133109C55
:104800000693F4E4DDF85CA0DDF850B0109CFFF7EF
:1048100058BB9A46069BBAF1390F03F10103029681
:10482000069306F10106D3D0B9F1000F3FF7DFAED2
:10483000E0E6249B022B3FF71AAE0697A5E5354626
:104840006BE7249B022B3FF712AE0F9B0697079353
:1048500017E54FF00209FFF75BBA024640F2EA2182
:10486000164B174803F0A2FA002520462946656436
:1048700001F038FB049078B900224FF4D5710F4B4A
:104880000F4803F093FA0F4B0493FFF700B93FF47E
:104890003FACC0F13C00BDE4049B012223644FF017
:1048A000FF3325950F930B920793FFF70ABB00BFC9
:1048B000000024400000E03F00001C40A8C20008A7
:1048C000BCC200089CC20008B1F90C20F8B50C4627
:1048D0001107074644D4636842F40062002BA281AA
:1048E0005CDDA56A002D57D000233E683B6093B283
:1048F00012F48052E16955D101233846A847421C81
:1049000066D0A389A56AE1695B0705D56368C01A0B
:10491000236B0BB1E36BC01A024600233846A8474D
:10492000451C48D13A68B4F90C30002A5CD01D2AE5
:1049300001D0162A3BD1002223F40063A38123690E
:10494000C4E90032216B3E6031B304F14003994267
:1049500002D0384600F076FA002318462363F8BDEB
:104960002669CEB193B2990718BF0023256808BF06
:1049700063692660AD1BA3600CE02B463246D4F879
:1049800024C03846E169E047B0F1000CA5EB0C0506
:10499000664409DD002DF0DC0020F8BDE36B002B40
:1049A0009FDCF9E7206DAFE74FF0FF30A38943F0BC
:1049B0004003A381F8BD0022B4F90C306260226983
:1049C00023F400632260DA04A381BBD52065B9E734
:1049D0003B68002B95D01D2B0FD0162B0DD0A38933
:1049E00043F04003A381F8BD23F4006362602269B1
:1049F000A381DB042260A5D5E8E700203E60F8BD76
:104A000038B505460C4608B1836BA3B1B4F90C0068
:104A1000B8B1636EDB0701D4810515D52846214660
:104A2000FFF752FF636E0546DA0702D4A3899B05A0
:104A30000ED5284638BD00F08FF8B4F90C000028D8
:104A4000E7D10546284638BDA06D00F015FDE5E725
:104A5000A06D00F019FD284638BD00BF38B548B339
:104A6000184B04461D680DB1AB6BBBB1B4F90C001B
:104A700088B1636EDB0701D4810513D52846214632
:104A8000FFF722FF636E0546DA0702D4A3899B0570
:104A90000CD5284638BD0546284638BD284600F0C6
:104AA0005BF8E3E7A06D00F0E7FCE7E7A06D00F03E
:104AB000EBFCEEE7044B05491868BDE8384000F010
:104AC0005DBC00BF140000202CC20008014A000891
:104AD000014900F053BC00BF957E000808B5436E45
:104AE000DA0702D483899B0501D5002008BD806DBB
:104AF00000F0C2FC002008BD08B5436EDA0702D4FE
:104B000083899B0501D5002008BD806D00F0BCFCA9
:104B1000002008BD682270B54D1E02FB05F50E464B
:104B200005F1740100F062FD044640B100210C3033
:104B3000C4E9016005F16802216001F075F92046C1
:104B400070BD00BF024B0349186800F017BC00BFDE
:104B50002CC20008957E00082DE9F04782463948AE
:104B600000F08AFCDAF83840002C66D104230322D6
:104B70003549DAF80450CAF83C10DFF8D090DFF875
:104B8000D080344F344E0AF53B71CAE9B921CAF8D6
:104B9000E0422146EB600822C5E90044C5E904442F
:104BA0006C66AC60AC6105F15C0001F03DF9C5E9F3
:104BB0000759C5E90987EE6205F1580000F054FC79
:104BC000DAF80850254B2146EB600822C5E900447D
:104BD000C5E904446C66AC60AC6105F15C0001F0B1
:104BE00023F9C5E90759C5E90987EE6205F15800BF
:104BF00000F03AFCDAF80C50194B2146EB60082221
:104C0000C5E90044C5E904446C66AC60AC6105F1DB
:104C10005C0001F009F905F15800C5E90759C5E93B
:104C20000A76C5F8248000F01FFC01230548CAF865
:104C30003830BDE8F04700F027BC0248BDE8F04737
:104C400000F022BC080A0020D14A0008D56D0008F7
:104C5000FD6D0008416E0008616E0008090001004A
:104C6000120002002DE9F04107462D4800F004FC37
:104C70002C4B1E68B36B93B34FF0040806F53876DF
:104C8000D6E90134013B04D525E05A1C04F168043F
:104C900021D0B4F90C50013B002DF6D1224B04F188
:104CA0005800E360656600F0DFFB1D4800F0ECFB98
:104CB00008222946C4E90155C4E904552560A561C7
:104CC00004F15C0001F0B0F8C4E90C55C4E91155D9
:104CD0002046BDE8F08135682DB12E46D0E730463C
:104CE000FFF73AFFC8E74FF4D671384600F07EFC74
:104CF000044668B1056029460546C0F804800C30BA
:104D00004FF4D072A06001F08FF834602E46B7E700
:104D10000348346000F0B8FB0C233B60D8E700BFC9
:104D2000040A00202CC200080100FFFF014800F027
:104D3000A3BB00BF040A0020014800F0A5BB00BFD0
:104D4000040A0020014800F097BB00BF080A0020B9
:104D5000014800F099BB00BF080A002008B50548CB
:104D600000F08AFB044B05491868BDE8084000F0D4
:104D7000E5BA00BF040A002014000020DD4A000844
:104D800008B5054B0549186800F0D8FABDE8084099
:104D9000034800F079BB00BF14000020F94A000866
:104DA000040A0020F8B50C46234F064601F08EF8A1
:104DB000BB685D68C4F57E6325F003050F332B44A3
:104DC00023F47F6323F00F03A3F58054B4F5805FD1
:104DD00007DB0021304601F0B3FFBB682B4498424B
:104DE00004D0304601F078F80020F8BD304661422A
:104DF00001F0A6FF01300DD0104ABB682D1B45F015
:104E000001055D60136830461B1B136001F064F8F8
:104E10000120F8BD0021304601F092FFBA68831AE4
:104E20000F2BDEDD43F001035360054B03491B6884
:104E3000C01A0860D5E700BFAC050020100A0020AA
:104E4000B409002000295FD0F8B50C46064601F0F1
:104E50003DF854F8043C764FA4F1080523F0010115
:104E60006818D7F808C04268844522F0030200F0B1
:104E70008680DB07426000EB020C33D454F8084C08
:104E8000DCF804302D1B2144AC6807F1080C6445A4
:104E900003F0010363D0D5F80CE0C4F80CE0CEF8C1
:104EA0000840002B00F08F8041F001036B6001602F
:104EB000B1F5007F31D24A09CB08012191407A68CF
:104EC00001331143796007EBC30257F83310083AF6
:104ED000C5E9021247F83350CD603046BDE8F840CE
:104EE00000F0FABFDCF80430DB070ED4114407F100
:104EF000080C836841F0010263456CD0C068D8603B
:104F000083606A606950D3E7704741F00103B1F5EF
:104F1000007F44F8043C0160CDD3B1F5206F4FEA27
:104F2000512345D28B0903F1390003F13802C30044
:104F3000F818FB580838984254D05A6822F00302F7
:104F40008A4202D99B689842F7D1D868C5E90230F5
:104F500085603046DD60BDE8F84000F0BDBF002B45
:104F600061D10A44D0E90213CB60996042F0010399
:104F70006B603046AA50BDE8F84000F0ADBF0A446F
:104F8000D90707D454F8083CED1A1A44D5E902139E
:104F9000CB60996042F001036B60264BBD601B68DB
:104FA00093429AD8244B30461968FFF7FBFE94E7EA
:104FB000142B0AD9542B1DD80B0B03F16F0003F1EE
:104FC0006E02C300B4E7114493E703F15C0003F100
:104FD0005B02C300ACE7C7E90455C5E902CC6A60CF
:104FE00069507AE70121921001FA02F279680A43C6
:104FF0007A60ABE7B3F5AA7F06D8CB0B03F1780054
:1050000003F17702C30093E740F25452934206D86B
:105010008B0C03F17D0003F17C02C30088E74FF4A1
:105020007E737E2284E741F001036B60016054E7E8
:10503000AC050020B8090020400A00209368002B2E
:1050400000F0F2802DE9F04FB1F90C3017461FFA4D
:1050500083FC1B0781460C4683B029D50B693BB303
:105060001CF002033D6832D04FF0000A5646D4F8D7
:1050700024B0E169DFF8C082B6B1464533465246F6
:1050800028BF43464846D847002840F3C380BB6842
:1050900082441B1A361ABB60002B00F0B180D4F892
:1050A00024B0E169002EE8D1D5E900A60835E3E790
:1050B00021464846FEF7AEFB002840F03A81B4F99D
:1050C0000C303D681FFA83FC1CF00203CCD11CF0AD
:1050D000010865D14646D4F808A02068002E5BD0B0
:1050E0001CF4007F00F0B780B245524600F2E68023
:1050F0001CF4906F32D06369216903EB430A0AEB19
:10510000DA7AA0EB010B731C4FEA6A0A5B44534541
:10511000524684BF9A4652461CF4806F00F0ED80E0
:105120001146484600F062FA002800F0FC805A461A
:105130002169019000F086FDA289019B22F4906212
:1051400042F08002A28103EB0B002361C4F814A09B
:10515000AAEB0B033246B246A3602060B34600269A
:105160004146019200F0E4FDA3682168019AA3EB97
:105170000A030A44A3602260B868D844A0EB0B007D
:10518000B86000283CD0B4F90CC0D4F808A020685E
:105190001FFA8CFC002EA3D1D5E9008608359DE7C7
:1051A000AA46984618461E461D46002E3ED00028A8
:1051B00046D0424620682169B24228BF3246884222
:1051C000636905D9A16803EB010B5A4500F386809A
:1051D000934276DC2A464846E169D4F824C0E04789
:1051E000B0F1000B16DDB8EB0B080DD00120BB6849
:1051F0005D44A3EB0B03A6EB0B06BB60002BD4D1E5
:10520000002003B0BDE8F08F21464846FFF7F8FBC9
:105210000028ECD0B4F90C304FF0FF3043F04003DD
:10522000A38103B0BDE8F08F002070470AF10803A6
:1052300053F8046C9A4653F8085C0833002EF7D0F4
:1052400032460A21284600F0B5FC002868D001301B
:10525000A0EB0508ADE72369834217D36369B34226
:1052600014D86FF0004CB44528BFB4469CFBF3FC47
:10527000424603FB0CF34846E169D4F824C0E047FA
:10528000B0F1000BC6DDA6EB0B0675E7B24528BFF3
:10529000B2464146524600F04BFDA3682268A3EB9C
:1052A0000A035244D346A3602260002BEBD121466F
:1052B0004846FFF7A5FB0028E5D0ABE7B2463246EB
:1052C0004CE729469346019200F032FDA368019A0B
:1052D0009B1AA36023681A44226084E729465A4631
:1052E00000F026FD236821465B4448462360FFF713
:1052F00087FB00283FF477AF8CE7484601F01EFBA0
:10530000034600287FF41FAF48462169FFF79AFD46
:105310000C22B4F90C30C9F8002023F080037BE79D
:10532000721C904646E70C22B4F90C30C9F80020F4
:1053300072E74FF0FF3064E700FCFF7F2DE9F0419A
:105340000026884600F53877D7E90154013D0ED490
:10535000A389013D012B06D9B4F90E30013302D0E7
:105360002046C04706436B1C04F16804F0D13F6837
:10537000002FE9D13046BDE8F08100BF2DE9F843A8
:105380004FF000090746884600F53876D6E9015403
:10539000013D10D4A389013D012B08D9B4F90E3089
:1053A000013304D021463846C04749EA00096B1C46
:1053B00004F16804EED13668002EE7D14846BDE816
:1053C000F88300BFF0307047004870473005002078
:1053D000004870473005002042B110B510460B4917
:1053E0001446FCF7BFFA18B9094810BD08487047C1
:1053F00020460749FCF7B6FA0028F5D020460549B3
:10540000FCF7B0FA0028EFD0002010BD00C3000860
:10541000FCC20008A0C40008014B93F828017047A3
:105420004004002041B110B508460C460A49FCF77B
:1054300099FA18B9094810BD08487047204607492D
:10544000FCF790FA0028F5D020460549FCF78AFAC7
:105450000028EFD0002010BD00C30008FCC20008E7
:10546000A0C40008704700BF704700BF704700BF6E
:10547000704700BF704700BF704700BF01207047F2
:1054800001207047704700BF704700BF2DE9F04111
:105490008B890C46990796B008D5012204F1430385
:1054A000C4E90432236016B0BDE8F081B4F90E10EF
:1054B0000646002927DB6A4602F03AFE002821DB77
:1054C000019D4FF4806805F47045A5F50055B5FAC7
:1054D00085F54FF400676D094146304600F086F8C7
:1054E000B4F90C30F0B1204A43F08003F263C4F801
:1054F0001480A3812060206135BB3B43A38116B09B
:10550000BDE8F081A38913F0800519D04FF0400861
:1055100030464146002500F069F82F46B4F90C30BA
:105520000028E0D19A05BED4012123F0030304F141
:10553000430243F00203C4E90421A3812260B2E7DD
:105540004FF480682F46C7E73046B4F90E1002F0DA
:1055500003FE10B9B4F90C30CFE7A38923F003039D
:1055600043F001031BB2C8E7D14A000870B50C46EE
:10557000B1F90E10154600291E4696B014DB6A4696
:1055800002F0D6FD00280FDB019A4FF4806302F48D
:105590007042A2F50052B2FA82F24FF40060520952
:1055A00032602B6016B070BD0023B4F90C1033606C
:1055B00011F0800004D0402218462A6016B070BD59
:1055C0004FF480632B6016B070BD00BF024B0146E4
:1055D000186800F00BB800BF14000020024B014611
:1055E0001868FFF72FBC00BF140000202DE9F04F12
:1055F00001F10B05162D064683B023D8102900F2C1
:10560000AE8000F063FC102518220220B64F3A4409
:105610005468A2F108039C4200F0AE806368E2681F
:10562000A16823F003032344CA6091605A6830469E
:1056300042F001025A60083400F04EFC204603B0EC
:10564000BDE8F08F35F0070500F18980A94200F22E
:10565000868000F03BFCB5F5FC7FC0F0A2816B0AB0
:1056600000F08480042B00F26E81AB0903F1390055
:1056700003F1380CC4009C4F3C446368083C9C42D6
:1056800006D10CE0002980F21F81DB689C4206D025
:105690005A6822F00302511B0F29F3DD60463C6972
:1056A000DFF848E2744572D0636823F0030CACEB7A
:1056B00005030F2B00F38581002BC7E904EE80F270
:1056C0007481BCF5007F80F01D8101224FEADC036C
:1056D0004FEA5C1C134402FA0CFC7A6807EBC30126
:1056E0004CEA020257F833C00839C4F808C0E16038
:1056F0007A6047F83340CCF80C404FF00108831033
:1057000008FA03F890454AD818EA020F08D120F0A9
:1057100003004FEA480818EA020F00F10400F8D02D
:1057200007EBC00A53468146D9680EE04A680C462A
:1057300022F00302A2EB050CBCF10F0FC96800F3C5
:105740000E81BCF1000F80F21F818B42EED109F176
:10575000010919F0030F03F10803E5D167E1002403
:105760000C232046336003B0BDE8F08F4FF4007483
:1057700040204FF03F0C7EE7D468A24208BF0230C1
:105780007FF44CAF3C69DFF864E174458CD14FF095
:1057900001087A68831008FA03F89045B4D9BC6808
:1057A000636823F003094D4503D8A9EB05030F2BCC
:1057B0007ADCDFF83CB14F4BDBF800201B6801328C
:1057C0002B4404EB090A00F04D8103F580530F339D
:1057D00023F47F6828F00F084146304601F0B0FA04
:1057E000411C024600F00881824500F20381424BD1
:1057F000196841440846196000F06A81DBF800101E
:10580000019301311BBFA2EB0A0A5044CBF80020E0
:10581000186012F0070B00F03281CBF108010A4446
:10582000CBF5805190440831A1EB0801C1F30B0A7C
:1058300051463046009201F083FA421CDDE9002314
:1058400000F06C81801A00EB0A08196848F001002A
:105850005144BC42BA601960506000F04581B9F112
:105860000F0F40F243814FF0050E6068A9F10C0C58
:105870002CF0070C00F0010040EA0C006060BCF165
:105880000F0F04EB0C00C0E901EE00F24F8114464B
:1058900050681A4B1A688A4238BF1960184B1A6848
:1058A0008A4238BF1960A9E0621943F0010345F04C
:1058B000010565603046BA600834536000F00CFBA7
:1058C000204603B0BDE8F08F1A44D3E90241E160FD
:1058D0008C605168304641F00101516003F10804C9
:1058E00000F0FAFAAAE600BFAC050020B4050020DB
:1058F000B4090020400A0020100A0020380A0020C5
:105900003C0A0020BCF5206F4FEA5C226BD3142ABE
:1059100000F2C68002F15C03DB005B32F918FB5831
:105920000839994200F0A1805A6822F003026245CA
:1059300002D99B689942F7D1D9687A68C4E90231E3
:105940008C60DC60D9E6142B66D9542B00F2B18050
:105950002B0B03F16F0003F16E0CC4008BE6304695
:10596000A668631945F001056560F1608E604CF032
:105970000101C7E90433C3E902EE596044F802C0EB
:1059800000F0AAFA083459E622445368304643F03E
:105990000103536054F8083FD9608B6000F09CFA13
:1059A0004CE6E80805F1080230E6A444DCF80430CF
:1059B000304643F00103CCF8043000F08DFA08348F
:1059C0003CE6621943F0010145F00105656030468F
:1059D000C7E90422C2E902EE516044F80C3000F03D
:1059E0007BFA08342AE64FEA9C1202F13903DB0005
:1059F000383293E7BC4266D0BC68606820F0030888
:105A00004545A8EB050302D80F2B3FF74DAF3046B5
:105A100000F062FA002411E603F15C0003F15B0C74
:105A2000C40028E65AF80839534540F09F8010F02A
:105A3000030F00F1FF30F5D17B6823EA08037B6098
:105A40004FEA480898453FF6AAAEB8F1000F04D1D6
:105A5000A5E64FEA480809F1040918EA030FF8D04F
:105A600048465DE603F11008B6E64FF0010C9210CF
:105A70000CFA02FC7A684CEA02027A605EE702EBFA
:105A800008014942C1F30B0A51463046009201F029
:105A900057F9431CDDE900237FF4D4AEDA46D4E69F
:105AA000542A26D84FEA1C3202F16F03DB006E3213
:105AB00034E7B3F5AA7F26D8EB0B03F1780003F1A6
:105AC000770CC400D7E52A4B18684044186095E667
:105AD000CAF30B0CBCF1000F7FF490AEBC68C84455
:105AE00048F001006060D4E61446D2E6012353601A
:105AF0008DE7B2F5AA7F24D84FEADC3202F17803B1
:105B0000DB0077320AE740F25452934224D8AB0CC0
:105B100003F17D0003F17C0CC400ACE5ABF1080B94
:105B2000D8444FF0000AA8EB02088EE604F1080101
:105B300030460093FFF786F9BC68009B60681968DF
:105B4000A7E640F254539A420CD84FEA9C4202F125
:105B50007D03DB007C32E1E64FF47E747F204FF062
:105B60007E0C88E54FF47E737E22D7E67B6867E77C
:105B7000100A002010B4034CD4F8E440A44610BC32
:105B8000604700BF4004002082B049B15AB16BB1F8
:105B900013780B601278101E18BF012002B07047F6
:105BA00001A9002AF3D1104602B070476FF001003E
:105BB000F4E700BF5FFA81FC810710D00346511E55
:105BC0002AB90AE09A0718460AD0013905D31846BF
:105BD00013F8012B6245F5D170470020704711463C
:105BE00003290CD80029F8D00346014401E08B4278
:105BF000F3D0184613F8012B6245F8D1ECE70246C2
:105C000010B54CEA0C2444EA0444104603680432FC
:105C10006340A3F1013E2EEA030313F0803F04D159
:105C2000043903291046F0D851B10346014401E07C
:105C30008B4205D0184613F8012B6245F8D110BDF0
:105C4000002010BD844641EA000313F0030349D14C
:105C5000403A23D30B6803604B6843608B688360D2
:105C6000CB68C3600B6903614B6943618B698361D6
:105C7000CB69C3610B6A03624B6A43628B6A8362BE
:105C8000CB6AC3620B6B03634B6B43638B6B8363A6
:105C9000CB6BC36340304031403ADBD230320BD360
:105CA0000B6803604B6843608B688360CB68C3609C
:105CB00010301031103AF3D20C3205D351F8043BB6
:105CC00040F8043B043AF9D2043208D0D2071CBF92
:105CD00011F8013B00F8013B01D30B8803806046BB
:105CE000704700BF082A13D38B07B1D010F003030D
:105CF000AED0C3F10403D21ADB071CBF11F8013B7D
:105D000000F8013BA4D331F8023B20F8023B9FE7A7
:105D1000043AD9D3013A11F8013B00F8013BF9D21A
:105D20000B7803704B7843708B78837060467047B4
:105D300088420DD98B1883420AD900EB020CBAB104
:105D4000624613F801CD994202F801CDF9D17047AE
:105D50000F2A0ED8034602F1FF3C4AB10CF1010CA8
:105D6000013B8C4411F8012B614503F8012FF9D157
:105D7000704740EA01039B074FD1A2F1100370B5B1
:105D800001F1200C23F00F0501F1100E00F11004B9
:105D9000AC441B095EF8105C0EF1100E44F8105C68
:105DA0005EF81C5C103444F81C5C5EF8185C44F827
:105DB000185C5EF8145CE64544F8145CEAD10133E3
:105DC00012F00C0F01EB031102F00F0400EB0313B0
:105DD00027D08E46043C24F003064FEA940C1E4460
:105DE0001C1F5EF8045B44F8045FB442F9D10CF167
:105DF000010402F0030203EB840301EB840102F1CE
:105E0000FF3C4AB10CF1010C013B8C4411F8012B11
:105E1000614503F8012FF9D170BD034602F1FF3C43
:105E20009CE72246EBE700BF830730B548D0541EFD
:105E3000002A3FD00346CAB201E0013C3AD303F83E
:105E4000012B9D07F9D1032C2DD9CDB245EA0525AB
:105E50000F2C45EA054536D9A4F1100222F00F0CAB
:105E600003F1200EE6444FEA121C03F1100242E94E
:105E7000045542E9025510327245F8D10CF1010285
:105E800014F00C0F03EB021204F00F0C13D0ACF162
:105E9000040323F003030433134442F8045B9342E6
:105EA000FBD10CF003042CB1CAB21C4403F8012B43
:105EB0009C42FBD130BD64461346002CF4D1F9E777
:105EC00003461446BFE71A46A446E0E70148FFF739
:105ED000D3BA00BF000A00200148FFF7D5BA00BFBF
:105EE000000A002038B5C36C05460C464BB153F888
:105EF000240080B1026843F824200023C0E9033362
:105F000038BD2122042101F077FF0346E864002810
:105F1000EDD1002038BD0121284601FA04F56A1DA3
:105F2000920001F069FF0028F3D0C0E90145E4E7E1
:105F300031B1C36C4A6853F82200086043F822105C
:105F4000704700BF2DE9F0414FF0000E0E461C4691
:105F50000D69074601F1140001680EF1010E8BB2C4
:105F600002FB0343090C4FEA134C02FB01CC9BB22A
:105F700003EB0C43754540F8043B4FEA1C44EBDC53
:105F80003CB1B368AB4207DD06EB850301355C61CC
:105F900035613046BDE8F081716838460131FFF760
:105FA000A1FF8046A8B1326906F10C0102329200CD
:105FB0000C30FFF747FEFB6C726853F8221031601B
:105FC00043F82260464606EB850301355C61356186
:105FD000DFE70246B521024B024801F0E7FE00BFB1
:105FE000A8C200080CC300082DE9F8431E46DFF8DC
:105FF000A0C0174603F108028CFB023C092E4FEAB1
:10600000E27305460C46C3EB6C0339DD4FF0010C1F
:1060100000214FEA4C0C634501F10101F9DC2846EF
:10602000FFF760FF014668B3089B092F43614FF0FB
:106030000103036112DC09270A34BE420BDDF61BA3
:10604000264414F8013B0A222846303BFFF77AFF2A
:10605000A6420146F5D10846BDE8F88304F10909D6
:10606000C8463C4418F8013B0A222846303BFFF75B
:1060700069FFA0450146F5D1A7F108044C44DCE7CF
:106080000021CCE70246CE21024B034801F08EFEF0
:10609000398EE338A8C200080CC30008020C1204B1
:1060A0000346CAB91020834013F07F4F04BF1B0280
:1060B000083013F0704F04BF1B01043013F0404F41
:1060C00004BF9B000230002B05DB13F0804F00F172
:1060D000010008BF202070470020E5E70368024662
:1060E00013F0070009D0D9071FD498074BBF5B08EE
:1060F0009B08012002201360704799B209B9102053
:10610000C340D9B209B908301B0A190704BF1B09DB
:106110000430990704BF9B080230D90703D45B08F9
:1061200000F1010003D01360704700207047202069
:10613000704700BF38B5C36C04460D464BB1586874
:10614000B0B102685A60002201234561C0E903230F
:1061500038BD2122042101F04FFE0346E0640028EF
:10616000EDD100224FF4A071074B084801F01EFE4C
:106170001C220121204601F03FFE0028F1D001221F
:106180000223C0E90123DEE7A8C200080CC300080F
:106190002DE9F04F0E6915698846AE42144685B068
:1061A00005DB2A46234635460C4616469846A36824
:1061B0006168AF19BB42B8BF0131FFF793FE019090
:1061C000002800F08780019B03F1140909EB870A7E
:1061D000D14505D24B46002243F8042B9A45FBD803
:1061E00008F1140808EB860B04F11403D8451A468D
:1061F00003EB85055FD22B1B153B23F00303043310
:106200001534A54238BF0423CDE902A7AC461F468A
:10621000924605E0000C29D1C34509F1040948D98B
:1062200058F8040B85B2002DF4D056464C46002396
:1062300056F8040B216882B21FFA81FE05FB02EEBC
:10624000000C0A0C05FB0022734402EB13429BB2C4
:1062500043EA0243B44544F8043B4FEA1243E7D80B
:1062600049F8073058F8040C000CD5D0D9F80030A4
:10627000544619464D4600222688090C00FB06119B
:106280009BB20A4443EA024345F8043B54F8046BCA
:106290002968360C8BB200FB0633A44503EB12438E
:1062A0004FEA1342E8D8C34549F8073009F1040919
:1062B000B6D8DDE902A7002F02DC05E0013F03D0DC
:1062C0005AF8043D002BF9D0019B18461F6105B018
:1062D000BDE8F08F024640F25D11024B024801F02A
:1062E00065FD00BFA8C200080CC3000812F003033C
:1062F0002DE9F041144607462ED10E46A4101CD0BD
:10630000BD6C95B3E3074FF0000806D4641014D0B9
:106310002868A8B10546E307F8D52A46314638462D
:10632000FFF736FFB6B17168FB6C641053F821209B
:10633000326043F821600646EAD13046BDE8F0817C
:106340002A4629463846FFF723FF28600546C0F84D
:106350000080E0E70646D9E70F4A013B52F82320C8
:106360000023FFF7EFFD0646C8E701213846FFF797
:10637000B9FD054640B140F271230122C0E9042372
:106380000023B8640360BDE702464FF4A071034BDD
:10639000034801F00BFD00BF68C40008A8C2000854
:1063A0000CC300082DE9F0470C462669A36806EBEC
:1063B0006216751C9D429046074649684FEA62196D
:1063C00004DD5B009D4201F10101FADC3846FFF774
:1063D00089FD002851D0B9F1000F00F114010FDD43
:1063E0000B464FF0000C09F105024FEA820E00EB5C
:1063F000820243F804CB9342FBD1AEF1140319445B
:10640000226904F1140318F01F0803EB820C2CD04E
:106410008E464FF0000AC8F120091A6802FA08F205
:1064200042EA0A024EF8042B53F8042B9C4522FA48
:1064300009FAF2D8ACEB0403153B23F00303043351
:1064400004F11502944538BF0423BAF1000F18BFB8
:106450002E4641F803A0FB6C6268066153F82210D7
:10646000216043F82240BDE8F087043953F8042B3B
:106470009C4541F8042FF9D8EDE7024640F2D911C6
:10648000014B024801F092FCA8C200080CC30008AE
:1064900084460B690069C01A15D10CF1140C143133
:1064A0000CEB830210B401EB830301E0944508D2A6
:1064B00052F8044D53F8041D8C42F7D004D24FF02B
:1064C000FF3010BC70477047012010BC704700BF00
:1064D0002DE9F84F0C6913698946E41A002C174618
:1064E0007DD101F11406143202EB830206EB830323
:1064F00001E09E4276D253F8045D52F8041D8D42AD
:10650000F7D067D3D9F80410FFF7ECFC002873D05C
:10651000D9F81050C46000F1140426464FF0000A68
:106520003B6909F1140807F1140E09F1100C08EB8E
:1065300085020EEB83095CF804BF5EF8041B1FFAAA
:106540008BF353441FFA81FA090CA3EB0A03C1EB46
:106550001B4101EB23419BB243EA0143F14546F85D
:10656000043B4FEA214AE6D8A9EB07011539153754
:10657000B94521F0030606F1040638BF042621F0D0
:10658000030138BF0021B044424526440C4418D9C9
:106590003746444654F8041B8BB253444FEA234A0F
:1065A0000AEB11419BB243EA0143A24247F8043B84
:1065B0004FEA214AEED8541EA4EB080424F0030449
:1065C000344423B954F8043D013D002BFAD0056151
:1065D000BDE8F88F4B460124B9461F4692E7F9DB28
:1065E00000248FE70021FFF77DFC60B1012200232A
:1065F000C0E90423BDE8F88F02464FF41071054B43
:10660000054801F0D3FB024640F23221014B02481B
:1066100001F0CCFBA8C200080CC300080F4B0B40D4
:10662000A3F15073002B02DD0020194670475B4236
:10663000B3F1A07F4FEA235205DA4FF40023002084
:1066400043FA02F17047143A1E2AD6BF4FF00043B6
:10665000012223FA02F20021104670470000F07F69
:106660002DE9F041076900F1140606EB87070C4697
:1066700057F8041CA7F104080846FFF70FFDC0F106
:1066800020030A28236034DD4645A0F10B001CD20C
:1066900057F8082C20B3C0F1200C814002FA00F01A
:1066A00022FA0CF21143A7F1080241F07F559642FD
:1066B00045F4401504D257F80C3C23FA0CF3184368
:1066C000044620462946BDE8F08140B101FA00F3B6
:1066D000002043F07F55044645F44015F1E702469B
:1066E000144641F07F5545F4401520462946BDE843
:1066F000F081C0F10B0321FA03F2464542F07F55C9
:106700002CBF002257F8082C45F4401538BFDA405A
:1067100000F1150301FA03F343EA02042046294677
:10672000BDE8F08170B5012182B016461D46FFF725
:10673000D9FB044600284CD02B46C5F30A55C3F3B9
:1067400013030DB143F48013002E019322D0684649
:106750000096FFF7C3FC002837D0019B0099C0F1D9
:10676000200203FA02F20A43C34001936261002B44
:1067700014BF02210121A3612161B5B1069BA5F2DD
:10678000334505441D60079BC0F135001860204665
:1067900002B070BD01A8FFF7A1FC0123019A1946C0
:1067A000626120302361002DE8D104EB8102A0F268
:1067B00032431069069A1360FFF770FCC0EB411179
:1067C0002046079B196002B070BDDDE900236261BD
:1067D000CDE7024640F20A31014B024801F0E6FAE9
:1067E000A8C200080CC300082DE9F04383B0884616
:1067F00069468146FFF734FF04460D46404601A92D
:10680000FFF72EFFD9F81030D8F810200F469A1A4B
:10681000DDE90063F31A03EB4213002B0CDD05EBFB
:10682000035906464D4632463B462046294602F06D
:10683000EFFA03B0BDE8F083C3EB033301EB035180
:1068400006460F46EFE700BF172870B506460ADD7B
:10685000002000240749084D22462B4602F0AEF9DD
:10686000013EF9D170BD054B03EBC006D6E900012E
:1068700070BD00BF0000F03F0000244078C3000856
:1068800001F1FF3C116902F114034FEA6C1C03EBA8
:1068900081010CF1010C8B4200EB8C0C16D210B56F
:1068A000A0F1040E53F8044B99424EF8044FF9D866
:1068B0008B1A153B23F0030304331844844504D991
:1068C000002340F8043B8445FBD810BD844505D91E
:1068D000002340F8043B8445FBD87047704700BF55
:1068E00003694A11934200F1140009DA00EB8303B3
:1068F00002E053F8042DAAB98342FAD80020704769
:1069000000EB8203F8DD11F01F01F5D010B450F850
:10691000224024FA01F202FA01F18C4208D001204F
:1069200010BC70470120704753F8042D002AF6D19F
:106930008342F9D8002010BC704700BF2DE9F84F02
:106940001646002900F09F8006F10B0507460C460D
:10695000FFF7BCFA162D5FD810252A46AE4260D844
:1069600054F804ECA4F108092EF00308904509EB53
:10697000080A63DAC24BDAF804009968514500F05E
:106980009A8020F0010353445B68DB076FD420F04A
:10699000030008EB0003934249DA1EF0010F11D106
:1069A00054F8083CA9EB030BDBF8041021F00301B9
:1069B00008444044904280F21A8108EB010393425C
:1069C00080F2ED8031463846FEF710FE0646E8B10B
:1069D00054F8043CA0F1080223F001034B44934215
:1069E00000F0D580A8F10402242A00F2FC80132ACA
:1069F000216800F2AE800346224619605168596052
:106A000092689A6021463846FEF71CFA3846FFF72E
:106A100063FA3046BDE8F88F25F00705002D2A46B9
:106A20009CDA0C2300263B603046BDE8F88F984680
:106A3000DAE9021209EB030ACA609160D9F804305E
:106A4000A8EB05020F2A03F0010321D848EA03034B
:106A5000C9F80430DAF8043043F00103CAF804300E
:106A600026463846FFF738FA3046BDE8F88F1EF064
:106A7000010FA7D154F8083CA9EB030BDBF8041075
:106A800021F0030199E71146BDE8F84FFEF7AEBDCE
:106A90002B4309EB050142F00102C9F804304A60BA
:106AA000DAF80430384643F001030831CAF80430FC
:106AB000FEF7C8F9D4E720F0030008EB000105F168
:106AC000100C614550DA1EF0010F7FF47BAF54F8D3
:106AD000081CA9EB010BDBF8041021F003010844AA
:106AE00000EB080AD4453FF768AF5E46DBF80C10B0
:106AF00056F8080FA8F10402242AC160886000F249
:106B0000E680132A216840F2E080CBF80810616823
:106B10001B2ACBF80C10A16800F2EB8008340BF1B3
:106B20001002116061685160A1689160AAEB0502D2
:106B30000BEB050142F0010299604A60DBF804307A
:106B4000384603F001031D43CBF80450FFF7C4F9A6
:106B50006AE7016063681B2A436070D8A16804F18A
:106B6000080200F1080348E7491B09EB050241F060
:106B700001019A60516054F8043C384603F0010367
:106B80001D4344F8045CFFF7A7F926464CE750F88C
:106B9000043C23F00303984409EB080A4EE75E46E1
:106BA000DBF80C1056F8080FA8F10402242AC16083
:106BB0000BEB030A886050D8132A21684BD9CBF815
:106BC000081061681B2ACBF80C10A1685AD8083449
:106BD0000BF11002116098466368D9465360A368B0
:106BE000344693602AE72146FFF7A2F80AE75E469B
:106BF000DAE90213CB60996056F8081FDBF80C3015
:106C0000A8F10402242ACB600BEB000A99602ED86D
:106C1000132A216829D9CBF8081063681B2ACBF8FE
:106C20000C3045D8A1680BF1100308341960626874
:106C300080465A60A268D94634469A60FEE6A36848
:106C4000242A8360E368C36028D0216904F110021C
:106C500000F11003D1E63246BCE7214630469846A3
:106C6000D946FFF765F83446E8E63346DEE72146C5
:106C700080463046D946FFF75BF83446DEE600BF73
:106C8000AC050020CBF81010E168242ACBF81410D2
:106C900023D021690BF1180210349BE7236904F11A
:106CA0001802036163694361A16900F11803A4E656
:106CB000A368242ACBF81030E368CBF8143024D032
:106CC00021690BF118031034B0E7324629E7214659
:106CD0003046FFF72DF8194B28E722691834CBF816
:106CE000182054F8042CCBF81C2021680BF120024A
:106CF00070E7CBF81010E168242ACBF8141010D0FC
:106D000021690BF1180210340BE723691834CBF812
:106D1000183054F8043CCBF81C3021680BF12003E8
:106D200084E722691834CBF8182054F8042CCBF8E7
:106D30001C2021680BF12002F3E600BFAC05002007
:106D4000002238B5064D044608462A6002F0B4FB1E
:106D5000431C00D038BD2B68002BFBD0236038BD0E
:106D6000440A0020F8B50027DFF85CC021F000439A
:106D7000634504460D46176023DC844653EA0C0C39
:106D80001FD0DFF848C0164601EA0C0C0A46BCF1D9
:106D9000000F09D100220E4B01F010FF6FF03507F4
:106DA00004460A4621F0004322F0FF421B1522F45C
:106DB000E002A3F2FE333B4442F07F55336045F4DA
:106DC000001520462946F8BDFFFFEF7F0000F07F49
:106DD0000000504310B50C46B1F90E1001F0E4F973
:106DE000002803DB236D0344236510BDA38923F42E
:106DF0008053A38110BD00BF00207047B1F90CC0C3
:106E00002DE9F0411CF4807F0C46054616461F46CE
:106E1000B1F90E100AD12CF4805C3B46324628466C
:106E2000A4F80CC0BDE8F04100F0AABF0223002284
:106E300001F0A4F9B4F90CC0B4F90E10EBE700BFEF
:106E400010B50C46B1F90E1001F098F9A389421C57
:106E50000EBF23F4805343F480532065A38110BDFB
:106E6000B1F90E1001F004B830B540EA0104A307EF
:106E700022D1032A20D90B468446194653F8045BD5
:106E8000A5F1013424EA050414F0803F15D1043A39
:106E9000032A19464CF8045BEFD801F1FF3E52B1CA
:106EA00063461EF8011F541E03F8011B41B1224620
:106EB0009C46002AF4D130BD844601F1FF3EEEE746
:106EC0006244002CF7D003F8011B9342FBD130BD84
:106ED0002DE9F84F4B6E90469C042DD593681268AF
:106EE00043B38B46064602F1080959E9025A5FEAA4
:106EF0009A0715D00024043D01E0A7420ED05A465F
:106F0000304655F8041F01F0A7F8431C04F10104B2
:106F1000F3D10023C8E90133BDE8F88FD8F8083071
:106F20002AF0030AA3EB0A03C8F8083009F108099C
:106F3000002BDAD10020ECE7FEF780F80023C8E947
:106F40000133BDE8F88F00BF10B4946814B110BCD1
:106F5000FFF7BEBF2046546010BC70472DE9F04FCC
:106F6000BDB01C460F461646CDE9053018B1836BFF
:106F7000002B00F072827B6EB7F90C10DD078AB22D
:106F800002D4900540F11E85930407D47B6E41F432
:106F9000005223F40053BA817B6692B2150740F188
:106FA000E3803B69002B00F0DF8002F01A030A2B1C
:106FB00000F0E78013AB10930023BB46CDE91133FB
:106FC000CDE90933CDE90B330DF14C090493337846
:106FD000002B00F0E581344604E014F8013F002B5B
:106FE00000F01581252BF8D1A51B40F013812378E3
:106FF000002B00F0D5814FF000038DF83B304FF0AF
:10700000FF3300254FF02B08019363780395661C2E
:107010000136A3F120025A2A00F22D81DFE812F096
:107020009B022B012B0197022B012B012B017702D5
:107030002B012B016B0267022B01630249022B011A
:1070400045025B005B005B005B005B005B005B007C
:107050005B005B002B012B012B012B012B012B0172
:107060002B012B012B010D026E002B012B012B019B
:107070002B012B012B012B012B012B012B01C50017
:107080002B012B012B01F1012B01B9022B012B014B
:1070900002052B012B012B012B012B012B012B01B5
:1070A0002B012B012B010D0270002B012B012B0159
:1070B000AF0270006A002B01A5022B013202C7004B
:1070C00020026A002B01F1016C0000052B012B014D
:1070D00022052B016C000021A3F1300216F8013BC0
:1070E00001EB810102EB4101A3F13002092AF5D93C
:1070F00003918EE745F02005337889E745F01005C8
:10710000AF0640F15D81059F073727F007073A4634
:107110007B6852F8087B98460592002BC0F23584B4
:10712000019B013300F01C8557EA080325F0800A13
:1071300000F010840A2F78F1000380F0BD84012351
:10714000554630378DF8EF7002930DF1EF049DF83E
:107150003B30DDE901829045B8BF9046002B00F03E
:107160009A8008F1010896E039460698FCF752FB30
:10717000002840F08085BA8902F01A030A2B7FF4B8
:1071800019AFB7F90E30002BFFF614AF7B6ED9079D
:1071900002D4930540F14F8523463246394606987E
:1071A0003DB0BDE8F04F00F091BD45F0100515F081
:1071B000200800F01681059F073727F007073B4698
:1071C000D7F8048053F8087B0593002325F4806AE0
:1071D0004FF000028DF83B20019A551C00F0EC8125
:1071E00057EA08012AF0800540F0E581002A40F0C6
:1071F000BA84002B40F0B3831AF00103029300F02D
:10720000DE8330230DF1EF048DF8EF309FE7A51BEF
:1072100000F0C680119B129A01332A44072BC9E95A
:1072200000651292119305DC09F10809049B2B44B7
:107230000493DCE6002A00F089835946069810AAD8
:10724000FFF746FE50B90DF14C09EFE75946069895
:1072500010AAFFF73DFE002800F09A805F467A6E84
:10726000BB89D10740F1A4805B0600F10D8504982D
:107270003DB0BDE8F08F002B00F092804FF0010888
:107280008DF88C304FF0000323AC8DF83B30CDF8F7
:1072900008800023019315F00203079318BF08F13B
:1072A0000208DDE9111215F0840701F10103184607
:1072B000089705D1039FA7EB0807002F00F38282F0
:1072C0009DF83B7009F1080C7FB1012101320DF1ED
:1072D0003B070728CDE91102C9E9007100F352828A
:1072E0000146E14601300CF1080C079BE3B1022393
:1072F0000232C9F8043007280FABCDE91102C9F8F2
:10730000003040F35982002A00F01983594606984C
:1073100010AAFFF7DDFD0028A0D1DDE911120DF163
:107320004C09481C0DF1540C089B802B00F07A810D
:10733000DDE90137DF1B002F00F3D381029B072813
:107340001A44CDE91102C9F80040C9F804300DDD36
:10735000002A00F086825946069810AAFFF7B8FD69
:1073600000287FF47BAF129A0DF14C0C680705D50D
:10737000039BA3EB0804002C00F37D82DDE90313DB
:107380004145ACBF5B1843440493002A7FF45EAFD1
:107390000023119333780DF14C09002B7FF41BAEC1
:1073A000129B5F46002B40F05C840023119356E74C
:1073B0009A053FF559AFB86DFEF766F8BB8953E7FC
:1073C000059AEC0602F1040300F10D836806059AA4
:1073D00040F10683B2F9007005934FEAE77843461F
:1073E0009BE6059915F0100201F1040340F00D83AE
:1073F00015F0400100F0E083059990460F88059351
:10740000E3E64FF00003059F8DF83B3057F8044B3F
:10741000019B002C00F0B183591C00F026831A4612
:1074200000212046FEF7C6FB002800F00984031B5C
:10743000029300230597019389E64FF000034FF074
:107440000108059F8DF83B3057F8043B23AC8DF8BD
:107450008C300597CDF808801BE7FDF77DFB8AE5AA
:1074600030228DF83C207822059B8DF83D2053F882
:10747000047BBD4A05934FF00008022345F0020A41
:107480000992A5E6059A52F8043B0592AA0600F176
:10749000B182EF0600F16D836C0600F1C083A80590
:1074A00040F16783049A1A7091E5337845F08005BE
:1074B000AEE5314611F8013B2A2B00F0EA83A3F137
:1074C0003002092A0E4600F2C1830023194616F83D
:1074D000013B01EB810102EB4101A3F13002092ADA
:1074E000F5D9019195E5337845F0040590E53378B9
:1074F0008DF83B808CE5059A337852F8041B0029FF
:1075000003910592BFF684AD4A420392ECE7069CD4
:107510002046FDF759FF436818460B93FAF700FB26
:10752000034620460C931C46FDF74EFF83680A93E2
:10753000002C3FF4E1AD0A9A3378002A3FF468AD9D
:107540001278002A3FF464AD45F4806560E5337835
:1075500045F001055CE59DF83B203378002A7FF477
:1075600057AD20228DF83B2052E533786C2B03BFBA
:10757000737845F02005013645F0100548E533786D
:10758000682B03BF737845F40075013645F040055C
:107590003EE545F0100A1AF0200800F0E681059F4C
:1075A0000123073727F007073A46D7F8048052F837
:1075B000087B05920CE6AA46012B3FF4BBAD022BDB
:1075C0003CAC12D1099A07F00F03D35C3F0947EA9C
:1075D00008774FEA181804F8013D57EA0803F2D17A
:1075E0003CAB1B1B55460293B1E507F00703FF08B0
:1075F00047EA48774FEAD808303357EA080122466D
:1076000004F8013DF1D11AF0010FE9D0302BE7D099
:107610003023023A04F8013C3CAB9B1A5546144611
:10762000029394E5039BA3EB0807002F7FF780AE3E
:10763000102FDFF838A133DDCC46B1462E46554633
:10764000A246069C06E0881C19460CF1080C103F67
:10765000102F1EDD10204B1C1032072BCDE91132EC
:10766000CCF80050CCF80400EDDD002A00F0858055
:107670005946204610AAFFF72BFC00287FF4EEADF8
:10768000DDE91112103F102F0DF14C0C01F101003A
:10769000E0DC5446AA4635464E46E1460CF1080C5D
:1076A0003A440728C9E900A7CDE9110240F39281C5
:1076B000002A00F0A0825946069810AAFFF708FC9D
:1076C00000287FF4CBADDDE90137DDE91112DF1BC6
:1076D000002F0DF14C0901F101000DF1540C7FF761
:1076E0002DAE102FDFF884A031DDCC46B1462E46FA
:1076F0005546A246069C06E0881C19460CF1080C6B
:10770000103F102F1CDD10204B1C1032072BCDE931
:107710001132CCF80050CCF80400EDDD42B35946EC
:10772000204610AAFFF7D4FB00287FF497ADDDE9CF
:107730001112103F102F0DF14C0C01F10100E2DC91
:107740005446AA4635464E46E1460CF1080C3A44EA
:107750000728C9E900A7CDE9110200F3DA80E14664
:1077600001300CF1080CE9E544C2000884C40008AB
:10777000012011460DF14C0CC2E7012011460DF11C
:107780004C0C64E7002A00F0D7805946069810AAEE
:10779000FFF79EFB00287FF461ADDDE911120DF1CA
:1077A0004C09481C0DF1540C9FE5022201200FAB3F
:1077B00013930DF1540C1492E1460146481C09F153
:1077C000080CB1E5102F40F34582DFF8E0A208462F
:1077D00051460D95B2465D460E46A346069C08E00E
:1077E00000F1020C184609F10809103F102F1CDDAA
:1077F000431C10211032072BCDE91132C9F800606B
:10780000C9F80410ECDD32B32946204610AAFFF770
:107810005FFB002840F09081DDE91102103F102F3E
:107820000DF14C0900F1010CE2DC3346604656468E
:107830009A465C46AB460D9D3A440728CDE91102B5
:10784000C9F800A0C9F8047000F3A980014609F145
:107850000809013034E510464FF0010C0DF14C09D8
:10786000C3E76C0711924CD5039BA3EB0804002CD3
:1078700047DD0DF14C0C102C119940F3EE81DFF82F
:107880002CA2B14610255646069F06E0881C1946D4
:107890000CF1080C103C102C19DD4B1C1032072B7E
:1078A000CCE90065CDE91132F0DD2AB359463846FE
:1078B00010AAFFF70DFB00287FF4D0ACDDE9111210
:1078C000103C102C0DF14C0C01F10100E5DCB2462E
:1078D0004E4622440728CCE900A4CDE911027FF7E7
:1078E0004DAD72B15946069810AAFFF7F1FA00287B
:1078F0007FF4B4AC129A41E5012011460DF14C0C15
:10790000C8E7DDE903234245ACBF9B184344049319
:107910003EE5002A00F013815946069810AAFFF7A9
:10792000D7FA00287FF49AAC1198129A0DF14C09FD
:1079300001300DF1540C01E5079B002B69D10120AA
:1079400011460DF14C090DF1540CEDE411920DF1BD
:107950004C096BE4019B002B7FF4F1AB55460023EF
:107960003CAC01930293FFF7F2BB05991AF01002A9
:1079700001F1040344D11AF0400100F0108105998F
:10798000904605930F88012322E42D237F428DF832
:107990003B30AA464FF0010368EB48081CE4002A7C
:1079A0006CD05946069810AAFFF792FA00287FF487
:1079B00055ACDDE911120DF14C09481C80E43CACDA
:1079C000FFF7C5BBB86DFDF757FDB7F90C108AB2CC
:1079D000FFF7DABA0146E14601300CF1080CA7E4E2
:1079E000A90500F12081176805934FEAE77843461F
:1079F000FFF793BB049A1A60D2175A60FFF7E7BAF1
:107A000005930F680123FFF7E3BB0F680593FFF7AA
:107A1000DCBB02220FAB13930DF154091492CDE697
:107A2000AA46B8E5224A099215F0200834D0059FED
:107A3000073727F007073A46D7F8048052F8087B43
:107A40000592EA0709D557EA080206D08DF83D30BD
:107A5000302345F002058DF83C30022325F4806A7E
:107A6000FFF7B6BB134A0992DEE720460597FAF7FF
:107A700057F80023CDE90130FFF769BB9DF83B10B3
:107A8000002900F0C08001220DF13B011046139146
:107A90000DF1540C149223E4059815F0100100F137
:107AA000040255D007680592CBE700BF74C40008F4
:107AB00058C2000844C2000800230AF48062CDF8CE
:107AC00008A0CDF81C90089699461646DDF828A027
:107AD0003CAD0CE00023384641460A2201F046FB4B
:107AE0000A2F78F100031BD30746884625463846FF
:107AF00041460A22002301F039FB30326C1E09F1A5
:107B0000010905F8012C002EE4D09AF800304B450D
:107B1000E0D1B9F1FF0FDDD00A2F78F1000355D283
:107B2000DDE90796CDF828A03CABDDF808A01B1BCB
:107B300055460293FFF70BBB2F46FFF790BB01237F
:107B4000029A13941193149212920DF1540C0DE4B5
:107B500015F040001AD0059888460788059270E70E
:107B6000AA46FFF7E7BA012BAA467FF428ADFFF734
:107B7000E6BA049A1A60FFF72ABA062B28BF062332
:107B8000494C984602930597FFF783BB059915F476
:107B900000781ABF80460F780F68059251E7059A62
:107BA0001AF40078059318BF88464FF0010314BFFC
:107BB00017781768FFF70CBB059A15F400781ABF01
:107BC0008846177817680593FFF7FFBA0C9B0B9947
:107BD000E41A1A462046FFF747F99AF801300BB12C
:107BE0000AF1010A384641460A2200234FF00009F3
:107BF00001F0BCFA78E7012011460DF14C090DF1B6
:107C0000540CFFF795BB079B002B7FF4CEAD1146BC
:107C100001200DF14C090DF1540CFFF789BB049ABA
:107C20001A80FFF7D4B992F9007005934FEAE7780C
:107C30004346FFF772BAB86DFDF726FCFFF7ACBA02
:107C4000019B059702930190FFF781BA00220192F0
:107C5000FFF7DFB9DFF854A0EEE5DFF850A0481CCD
:107C600037E65946069810AAFFF732F900283FF484
:107C70009CABFFF7F4BA7B6EDC0705D4BB89980593
:107C800002D4B86DFDF700FC4FF0FF330493FFF70B
:107C9000EEBA059A73780E4652F8041B059241EA33
:107CA000E1720192FFF7B4B96CC2000874C4000815
:107CB0008C4600B586461346034A714610685DF847
:107CC00004EB6246FFF74AB914000020F0B54FF408
:107CD000806C1546002406461F46ADF26C4D1AAB6B
:107CE000009304938B8916A823F00203ADF80C309F
:107CF0004B6E06941993CB890C46ADF80E30CB69C8
:107D0000CDF808C007934B6ACDF814C00993FDF76E
:107D1000ABFB2A463B4669463046FFF71FF9051E76
:107D200007DB69463046FCF76BFE002818BF4FF0B2
:107D3000FF35BDF80C305B0603D5A38943F0400343
:107D4000A3811698FDF794FB28460DF26C4DF0BD0B
:107D500010B4034CD4F8E040A44610BC604700BF08
:107D600040040020034649B1FF2A02D801200A70CE
:107D700070478A224FF0FF301A60704708467047FC
:107D800038B50C46114600228446074D20462A602D
:107D90001A466446F9F76EFA431C00D038BD2B68CA
:107DA000002BFBD0236038BD440A0020144600B5E8
:107DB0001A460A4B0D461B6885B0DE6803464CB177
:107DC00007490191304607490294009500F0E0F818
:107DD00000F0AAFA04490C46F3E700BF14000020A3
:107DE00094C40008A4C40008A0C4000808B5134641
:107DF0000022FFF7DBFF00BF38B5A1FB021484BBF4
:107E0000FDF7F4FB0546D8B150F8042C22F003022C
:107E1000043A242A16D8132A19D91B2AC0E9004487
:107E20001CD90023242A14BF00F1100200F118020B
:107E3000C0E9024404BF04614461C2E900339360B5
:107E4000284638BD2146FDF7EFFF284638BD0246DB
:107E500000232846C2E90033936038BD00F10802D0
:107E6000F6E7F9F7A3FB0C2300250360E8E700BF62
:107E7000002238B5064D044608462A6001F0E4FAAF
:107E8000431C00D038BD2B68002BFBD0236038BDCD
:107E9000440A002070B500294AD005460C4610B1AE
:107EA000836B002B47D0636EB4F90C20D80732D512
:107EB000002A3DD021462846FCF706FDE36A064627
:107EC00033B12846E16998470028B8BF4FF0FF3624
:107ED000A3891A063CD4216B41B104F140039942B5
:107EE00002D02846FCF7AEFF00232363616C21B16A
:107EF0002846FCF7A7FF00236364FCF717FF002266
:107F0000636EA281DB0728D5A06DFDF7B1FAFCF7FF
:107F100013FF304670BD9105CCD4A06DFDF7ACFACF
:107F2000B4F90C30002BC5D1666E16F001060AD0EC
:107F30000026304670BDFCF70FFE636EB4F90C20CE
:107F4000D807B5D4E7E7A06DFDF79EFA304670BDBF
:107F500028462169FCF776FFBDE7A06DFDF794FA8E
:107F6000D2E700BF024B01461868FFF793BF00BF7E
:107F7000140000200CB400B583B004AB53F8042BFC
:107F80000193FEF7EBFF03B05DF804EB02B070471E
:107F90000EB400B5074A82B003AB0146106853F82F
:107FA000042B0193FEF7DAFF02B05DF804EB03B097
:107FB000704700BF140000202DE9F04383B007464E
:107FC00088461446FDF728FA012803D108F1FF334B
:107FD000FE2B33D94246384604F15C0301A900F078
:107FE00065F9421C06462FD018B39DF804100025F1
:107FF0000DF1050908E023685A1C2260197001354B
:10800000B54216D219F8011BA368013B002BA360EF
:10801000F1DAA269934201DB0A29ECD12246384603
:10802000FBF796FB431CEAD10646304603B0BDE899
:10803000F0834646304603B0BDE8F0835FFA88F12E
:1080400006468DF80410D2E73046A38943F040037A
:10805000A38103B0BDE8F08330B514460546606ED9
:10806000B2F90C30C00783B09AB201D490051CD588
:10807000900406D4626E43F4005342F40052A3818C
:10808000626622462846FFF797FF636E0546DA07C9
:1080900002D4A3899B0502D5284603B030BDA06D4C
:1080A000FDF7F2F9284603B030BDA06D0191FDF750
:1080B000E3F9B4F90C3001999AB2D9E71B4B70B5CA
:1080C0001E6805460C460EB1B36BF3B1616EB4F990
:1080D0000C30C9079AB201D490051FD5910406D47B
:1080E000626E43F4005342F40052A381626622465A
:1080F00029463046FFF760FF636E0546DA0702D473
:10810000A3899B0505D5284670BD3046FCF724FDA4
:10811000DCE7A06DFDF7B8F9284670BDA06DFDF74E
:10812000ABF9B4F90C309AB2D8E700BF14000020C4
:1081300070B50026074D0446084611462E6001F032
:108140008BF9431C00D070BD2B68002BFBD0236043
:1081500070BD00BF440A0020002238B5064D044619
:1081600008462A6001F088F9431C00D038BD2B680E
:10817000002BFBD0236038BD440A002038B50C46E4
:10818000114600228446074D20462A601A4664465E
:1081900001F082F9431C00D038BD2B68002BFBD0C6
:1081A000236038BD440A002038B50C461146002231
:1081B0008446074D20462A601A46644601F074F949
:1081C000431C00D038BD2B68002BFBD0236038BD8A
:1081D000440A00202DE9F0410E680C460546BEB168
:1081E00037688FB1D7F80080B8F1000F08D0D8F801
:1081F000001009B1FFF7EEFF41462846FCF722FECA
:1082000039462846FCF71EFE31462846FCF71AFE82
:1082100021462846BDE8F041FCF714BE224B1B68FE
:10822000834240D0C16C70B5054681B100268C599F
:108230003CB1214624682846FCF704FE002CF8D106
:10824000E96C0436802EF2D12846FCF7FBFD296C40
:1082500011B12846FCF7F6FDD5F8484154B105F5B3
:10826000A676B44206D0214624682846FCF7EAFDEB
:10827000A642F8D1696D11B12846FCF7E3FDAB6B5E
:1082800083B12846EB6B9847D5F8E04254B121689A
:1082900011B12846FFF79EFF21462846BDE87040F1
:1082A000FCF7D0BD70BD70471400002070B50B4CBA
:1082B0001E46D4F8E05084B0044621B1A847431CC0
:1082C00006D004B070BD0A4601A9A847431CF8D1E6
:1082D00000228A233260236004B070BD4004002075
:1082E00070B50F4B0F4CD3F8E06025680B46144671
:1082F000014684B038B11A4628462346B047431C8D
:1083000008D004B070BD134601A902462846B04704
:10831000431CF6D100228A2322602B6004B070BD7A
:108320004004002014000020062008B500F0A2F848
:10833000012001F0CFF800BF38B5D0F8DC420CB115
:10834000002038BD80210546FDF750F90246C5F8EA
:10835000DC0230B1031F7C3243F8044F9342FBD15F
:10836000EEE74FF0FF3038BD1F29F8B5054609D8B4
:10837000D0F8DC620C4617464EB156F8240046F899
:108380002470F8BD16234FF0FF302B60F8BD80211C
:10839000FDF72CF90646C5F8DC0240B10021031FA9
:1083A00000F17C0543F8041F9D42FBD1E5E74FF047
:1083B000FF30F8BD1F2938B5054621D8D0F8DC229A
:1083C0000C466AB152F8213053B1012B16D0591C1A
:1083D00010D00025204642F824509847284638BD42
:1083E000284600F003F9224601462846BDE83840F9
:1083F00000F0E8B8162301202B6038BD002038BDFE
:1084000016234FF0FF302B6038BD00BF1F292DD839
:10841000D0F8DC2238B50C46054682B152F824303B
:1084200002EB84024BB1591C1BD0012B17D0002545
:10843000204615609847284638BD012038BD802168
:10844000FDF7D4F80246C5F8DC0260B10020131F26
:1084500002F17C0143F8040F9942FBD1DEE70320CF
:1084600038BD022038BD4FF0FF3038BD4FF0FF302F
:10847000704700BF38B5154B1F281D6820D8D5F8A8
:10848000DC22044662B152F820304BB1012B15D0EA
:10849000591C0FD0002542F820509847284638BD77
:1084A000284600F0A3F8224601462846BDE8384099
:1084B00000F088B8162301202B6038BD002038BD9D
:1084C00016234FF0FF302B6038BD00BF1400002092
:1084D000134B1F2870B51E6809D80D46D6F8DC125C
:1084E000044649B151F8240041F8245070BD1623C8
:1084F0004FF0FF30336070BD80213046FDF776F8D5
:108500000146C6F8DC0240B10022031F00F17C0CDA
:1085100043F8042F6345FBD1E4E74FF0FF3070BD13
:108520001400002038B50C4B1D68D5F8DC420CB1A6
:10853000002038BD80212846FDF758F8C5F8DC0238
:1085400038B1031F00F17C0243F8044F9342FBD182
:10855000EEE74FF0FF3038BD1400002038B5184B5F
:108560001F281D6829D8D5F8DC22044682B152F8AC
:10857000243002EB84024BB1591C1CD0012B18D0C3
:108580000025204615609847284638BD012038BD93
:1085900080212846FDF72AF80246C5F8DC0260B1C2
:1085A0000020131F02F17C0143F8040F8B42FBD122
:1085B000DDE7032038BD022038BD4FF0FF3038BD65
:1085C0001400002070B50026074D044608461146E9
:1085D0002E6000F059FF431C00D070BD2B68002BAB
:1085E000FBD0236070BD00BF440A002000F03CBFF8
:1085F00070B54FF0FF0C4CF4E06C1CEA11541DBF39
:108600001CEA135594EA0C0F95EA0C0F00F0DEF803
:108610002C4481EA030621EA4C5123EA4C5350EAE8
:10862000013518BF52EA033541F4801143F4801339
:1086300038D0A0FB02CE4FF00005E1FB02E506F0CA
:108640000042E0FB03E54FF00006E1FB03569CF01F
:10865000000F18BF4EF0010EA4F1FF04B6F5007F25
:1086600064F5407404D25FEA4E0E6D4146EB060697
:1086700042EAC62141EA55514FEAC52040EA5E5020
:108680004FEACE2EB4F1FD0C88BFBCF5E06F1ED8CA
:10869000BEF1004F08BF5FEA500E50F1000041EB01
:1086A000045170BD06F0004646EA010140EA0200AE
:1086B00081EA0301B4EB5C04C2BFD4EB0C0541EAD0
:1086C000045170BD41F480114FF0000E013C00F3E5
:1086D000AB8014F1360FDEBF002001F0004170BD09
:1086E000C4F10004203C35DA0C341BDC04F1140422
:1086F000C4F1200500FA05F320FA04F001FA05F2AE
:1087000040EA020001F0004221F0004110EBD3707A
:1087100021FA04F642EB06015EEA430E08BF20EAA6
:10872000D37070BDC4F10C04C4F1200500FA04F349
:1087300020FA05F001FA04F240EA020001F00041DB
:1087400010EBD37041F100015EEA430E08BF20EA4E
:10875000D37070BDC4F1200500FA05F24EEA020E96
:1087600020FA04F301FA05F243EA020321FA04F0C5
:1087700001F0004121FA04F220EA020000EBD3707C
:108780005EEA430E08BF20EAD37070BD94F0000F7C
:108790000FD101F00046400041EB010111F4801FB0
:1087A00008BF013CF7D041EA060195F0000F18BF61
:1087B000704703F00046520043EB030313F4801F9D
:1087C00008BF013DF7D043EA0603704794EA0C0F57
:1087D0000CEA135518BF95EA0C0F0CD050EA41066D
:1087E00018BF52EA4306D1D181EA030101F00041EA
:1087F0004FF0000070BD50EA410606BF1046194612
:1088000052EA430619D094EA0C0F02D150EA01361D
:1088100013D195EA0C0F05D152EA03361CBF10465E
:1088200019460AD181EA030101F0004141F0FE41FD
:1088300041F470014FF0000070BD41F0FE4141F481
:10884000780170BD81F0004102E000BF83F0004379
:1088500030B54FEA41044FEA430594EA050F08BFDB
:1088600090EA020F1FBF54EA000C55EA020C7FEA9F
:10887000645C7FEA655C00F0E2804FEA5454D4EB1C
:108880005555B8BF6D420CDD2C4480EA020281EAE6
:10889000030382EA000083EA010180EA020281EA1E
:1088A0000303362D88BF30BD11F0004F4FEA013170
:1088B0004FF4801C4CEA113102D0404261EB41017F
:1088C00013F0004F4FEA03334CEA133302D0524205
:1088D00063EB430394EA050F00F0A780A4F10104C1
:1088E000D5F1200E0DDB02FA0EFC22FA05F28018FB
:1088F00041F1000103FA0EF2801843FA05F35941E1
:108900000EE0A5F120050EF1200E012A03FA0EFC5F
:1089100028BF4CF0020C43FA05F3C01851EBE37189
:1089200001F0004507D54FF0000EDCF1000C7EEBA6
:1089300000006EEB0101B1F5801F1BD3B1F5001FE4
:108940000CD349085FEA30004FEA3C0C04F1010403
:108950004FEA445212F5800F80F09A80BCF1004F2C
:1089600008BF5FEA500C50F1000041EB045141EAAE
:10897000050130BD5FEA4C0C404141EB0101013C77
:1089800028BFB1F5801FE9D291F0000F04BF014666
:108990000020B1FA81F308BF2033A3F10B03B3F138
:1089A00020020CDA0C3208DD02F1140CC2F10C02C8
:1089B00001FA0CF021FA02F10CE002F11402D8BF26
:1089C000C2F1200C01FA02F120FA0CFCDCBF41EAF2
:1089D0000C019040E41AA2BF01EB0451294330BDC1
:1089E0006FEA04041F3C1CDA0C340EDC04F114049E
:1089F000C4F1200220FA04F001FA02F340EA030075
:108A000021FA04F345EA030130BDC4F10C04C4F1BA
:108A1000200220FA02F001FA04F340EA030029469A
:108A200030BD21FA04F0294630BD94F0000F83F4E4
:108A3000801306BF81F480110134013D4EE77FEAC7
:108A4000645C18BF7FEA655C29D094EA050F08BF13
:108A500090EA020F05D054EA000C04BF19461046F4
:108A600030BD91EA030F1EBF0021002030BD5FEA38
:108A7000545C05D14000494128BF41F0004130BD60
:108A800014F580043CBF01F5801130BD01F00045B4
:108A900045F0FE4141F470014FF0000030BD7FEA27
:108AA000645C1ABF194610467FEA655C1CBF0B4622
:108AB000024650EA013406BF52EA033591EA030F39
:108AC00041F4002130BD00BF90F0000F04BF002131
:108AD000704730B54FF4806404F132044FF0000564
:108AE0004FF0000150E700BF90F0000F04BF0021DD
:108AF000704730B54FF4806404F1320410F0004543
:108B000048BF40424FF000013EE700BF42004FEA3D
:108B1000E2014FEA31014FEA02701FBF12F07F43BA
:108B200093F07F4F81F06051704732F07F4208BF71
:108B3000704793F07F4F04BF41F40021704730B578
:108B40004FF4607401F0004521F000411CE700BFC4
:108B500050EA010208BF704730B54FF000050AE047
:108B600050EA010208BF704730B511F0004502D548
:108B7000404261EB41014FF4806404F132045FEA4A
:108B8000915C3FF4D8AE4FF003025FEADC0C18BFF3
:108B900003325FEADC0C18BF033202EBDC02C2F1E5
:108BA000200300FA03FC20FA02F001FA03FE40EA77
:108BB0000E0021FA02F11444BDE600BF70B54FF07B
:108BC000FF0C4CF4E06C1CEA11541DBF1CEA135559
:108BD00094EA0C0F95EA0C0F00F0DEF82C4481EAC1
:108BE000030621EA4C5123EA4C5350EA013518BFE1
:108BF00052EA033541F4801143F4801338D0A0FBCE
:108C000002CE4FF00005E1FB02E506F00042E0FB7A
:108C100003E54FF00006E1FB03569CF0000F18BF80
:108C20004EF0010EA4F1FF04B6F5007F64F5407428
:108C300004D25FEA4E0E6D4146EB060642EAC621BB
:108C400041EA55514FEAC52040EA5E504FEACE2E28
:108C5000B4F1FD0C88BFBCF5E06F1ED8BEF1004F2B
:108C600008BF5FEA500E50F1000041EB045170BDA7
:108C700006F0004646EA010140EA020081EA0301EB
:108C8000B4EB5C04C2BFD4EB0C0541EA045170BDE7
:108C900041F480114FF0000E013C00F3AB8014F161
:108CA000360FDEBF002001F0004170BDC4F10004AA
:108CB000203C35DA0C341BDC04F11404C4F120052B
:108CC00000FA05F320FA04F001FA05F240EA020086
:108CD00001F0004221F0004110EBD37021FA04F6BC
:108CE00042EB06015EEA430E08BF20EAD37070BD76
:108CF000C4F10C04C4F1200500FA04F320FA05F0D5
:108D000001FA04F240EA020001F0004110EBD370D6
:108D100041F100015EEA430E08BF20EAD37070BD46
:108D2000C4F1200500FA05F24EEA020E20FA04F31F
:108D300001FA05F243EA020321FA04F001F00041CE
:108D400021FA04F220EA020000EBD3705EEA430E3F
:108D500008BF20EAD37070BD94F0000F0FD101F06E
:108D60000046400041EB010111F4801F08BF013CA7
:108D7000F7D041EA060195F0000F18BF704703F0E5
:108D80000046520043EB030313F4801F08BF013D6C
:108D9000F7D043EA0603704794EA0C0F0CEA135528
:108DA00018BF95EA0C0F0CD050EA410618BF52EAE2
:108DB0004306D1D181EA030101F000414FF00000E8
:108DC00070BD50EA410606BF1046194652EA4306F6
:108DD00019D094EA0C0F02D150EA013613D195EA6A
:108DE0000C0F05D152EA03361CBF104619460AD1B2
:108DF00081EA030101F0004141F0FE4141F47001BC
:108E00004FF0000070BD41F0FE4141F4780170BDAB
:108E100070B54FF0FF0C4CF4E06C1CEA11541DBF10
:108E20001CEA135594EA0C0F95EA0C0F00F0A7F812
:108E3000A4EB050481EA030E52EA03354FEA01313F
:108E400000F088804FEA03334FF0805545EA131352
:108E500043EA12634FEA022245EA111545EA10651A
:108E60004FEA00260EF000419D4208BF964244F1B1
:108E7000FD0404F5407402D25B084FEA3202B61AD0
:108E800065EB03055B084FEA32024FF480104FF4A4
:108E9000002CB6EB020E75EB030E22BFB61A754618
:108EA00040EA0C005B084FEA3202B6EB020E75EBAB
:108EB000030E22BFB61A754640EA5C005B084FEA13
:108EC0003202B6EB020E75EB030E22BFB61A7546E0
:108ED00040EA9C005B084FEA3202B6EB020E75EBEB
:108EE000030E22BFB61A754640EADC0055EA060EAC
:108EF00018D04FEA051545EA16754FEA06164FEAEF
:108F0000C30343EA52734FEAC2025FEA1C1CC0D19A
:108F100011F4801F0BD141EA00014FF000004FF027
:108F2000004CB6E711F4801F04BF01430020B4F1E8
:108F3000FD0C88BFBCF5E06F3FF6AFAEB5EB030CA0
:108F400004BFB6EB020C5FEA500C50F1000041EB9D
:108F5000045170BD0EF0004E4EEA113114EB5C046A
:108F6000C2BFD4EB0C0541EA045170BD41F480113D
:108F70004FF0000E013C90E645EA060E8DE60CEA45
:108F8000135594EA0C0F08BF95EA0C0F3FF43BAF62
:108F900094EA0C0F0AD150EA01347FF434AF95EA19
:108FA0000C0F7FF425AF104619462CE795EA0C0FFD
:108FB00006D152EA03353FF4FDAE1046194622E7CA
:108FC00050EA410618BF52EA43067FF4C5AE50EAA4
:108FD00041047FF40DAF52EA43057FF4EBAE12E794
:108FE0004FF0FF3C06E000BF4FF0010C02E000BF75
:108FF0004FF0010C4DF804CD4FEA410C7FEA6C5C58
:109000004FEA430C18BF7FEA6C5C1BD001B050EAFA
:10901000410C0CBF52EA430C91EA030F02BF90EAE5
:10902000020F0020704710F1000F91EA030F58BFA4
:10903000994208BF90422CBFD8176FEAE37040F006
:10904000010070474FEA410C7FEA6C5C02D150EAA4
:10905000013C07D14FEA430C7FEA6C5CD6D152EA5F
:10906000033CD3D05DF8040B704700BF8446104624
:1090700062468C461946634600E000BF01B5FFF723
:10908000B7FF002848BF10F1000F01BD4DF808EDF3
:10909000FFF7F4FF0CBF012000205DF808FB00BFC4
:1090A0004DF808EDFFF7EAFF34BF012000205DF81E
:1090B00008FB00BF4DF808EDFFF7E0FF94BF01206B
:1090C00000205DF808FB00BF4DF808EDFFF7CEFF6C
:1090D00094BF012000205DF808FB00BF4DF808EDAB
:1090E000FFF7C4FF34BF012000205DF808FB00BF7C
:1090F0004FEA410C7FEA6C5C02D150EA013C0AD194
:109100004FEA430C7FEA6C5C02D152EA033C02D185
:109110004FF0000070474FF0010070474FEA4102E6
:1091200012F5001215D211D56FF47873B3EB6252B9
:1091300012D94FEAC12343F0004343EA505311F0E0
:10914000004F23FA02F018BF404270474FF0000072
:10915000704750EA013005D111F0004008BF6FF0B0
:10916000004070474FF00000704700BF53B94AB944
:10917000002908BF00281CBF4FF0FF314FF0FF301F
:1091800000F060B9ADF1080C6DE904CE00F006F80E
:10919000DDF804E0DDE9022304B070472DE9F04F6B
:1091A00007468C46084615463C461946099E002B44
:1091B00040F0C6808242B2FA82F746D94FB1C7F179
:1091C000200E24FA0EFE00FA07F3BD404EEA030C0F
:1091D000BC404FEA1548BCFBF8F91FFA85FE08FBB6
:1091E00019C309FB0EFA220C42EA03439A4528D917
:1091F000EB1809F1FF3004D29A4502D9A9F1020017
:109200002B44A3EB0A03B3FBF8F208FB123302FB77
:109210000EFEA4B244EA0344A64514D92C1902F167
:10922000FF3303D2A64501D9931E2C44A4EB0E04B0
:1092300043EA00401EB10023FC4034607360BDE887
:10924000F08F4846DDE71346F0E702B9FFDE87BB43
:109250000121831A4FEA154EB3FBFEFCAAB20EFBA6
:109260001C330CFB02F8200C40EA0343984563D9F9
:10927000EB180CF1FF3004D2984502D9ACF1020092
:109280002B44A3EB0803B3FBFEFC0EFB1C330CFBCF
:1092900002F2A4B244EA0344A2424FD92C190CF1C1
:1092A000FF3304D2A24202D9ACF102032C44A41A27
:1092B000BEE7C7F1200CBD4020FA0CF800FA07F316
:1092C00024FA0CFC4FEA154E4CEA0302B8FBFEFCF4
:1092D000ABB20EFB1C800CFB03F9110C41EA004001
:1092E000814504FA07F423D928180CF1FF3104D280
:1092F000814502D9ACF102012844A0EB0900B0FB82
:10930000FEFC0EFB1C000CFB03F892B242EA004389
:1093100098450FD9EB180CF1FF3204D2984502D9C9
:10932000ACF102022B44A3EB080342EA014191E7AE
:109330006146E2E76246F6E76046A2E76346B6E7C3
:10934000834205D90EB1C6E900700021084676E7D0
:10935000B3FA83F181B9834201D3BA420AD8BC1A65
:1093600060EB030301209C46002E68D0C6E9004C48
:10937000002164E70846F7E7C1F1200C8B4022FA90
:109380000CF41C4320FA0CFB4FEA1449BBFBF9F820
:109390001FFA84FE09FB18BB08FB0EFA02FA01F55E
:1093A00000FA01F327FA0CF213431A0C42EA0B42BB
:1093B000924507FA01F73ED9A21808F1FF3004D20E
:1093C000924502D9A8F102002244A2EB0A02B2FBA4
:1093D000F9F809FB182208FB0EFE9BB243EA024291
:1093E00096452AD9A21808F1FF3304D2964502D92E
:1093F000A8F10203224443EA0040A0FB0593A2EB3C
:109400000E029A42CE46984602D306D14F4504D268
:10941000B9EB050E63EB0408013886B1B7EB0E0318
:1094200062EB080707FA0CFCCB404CEA0303CF4081
:10943000C6E900379CE74046C7E74346DBE73146CD
:10944000FDE60000704700BF5822024B4FF0FF308E
:109450001A607047440A00205822024B4FF0FF3038
:109460001A607047440A00205822024B4FF0FF3028
:109470001A607047440A00205822024B00201A60EC
:10948000704700BF440A00205822024B4FF0FF30C3
:109490001A607047440A00205822024B4FF0FF30F8
:1094A0001A607047440A00205822024B4FF0FF30E8
:1094B0001A607047440A0020044A05491368002BCB
:1094C00008BF0B461844106018467047480A002031
:1094D0004C0A0020FEE700BF024A936843F00103F4
:1094E0009360704700300240014B18601868704765
:1094F00000300240002310B5044A8B4201DB1068A3
:1095000010BD50F8234001331460F6E700300240EC
:10951000014BB3F8E007704700F0FF1F054BD3F88D
:10952000F0270260D3F8EC274260D3F8E837836075
:10953000704700BF00F0FF1F024A136843F00803A2
:109540001360704700200240024A136823F00803AA
:10955000136070470020024008B5FFF7D9FFB0F54F
:10956000007F09D9054B1A6D42F080021A65044A42
:109570005A6402F188325A6408BD00BF00200240DC
:1095800023016745024A136D43F08003136570475A
:109590000020024008B5FFF7BBFFB0F5007F81BF98
:1095A000024AD36C43F00403D36408BD0020024098
:1095B00008B5FFF7ADFFB0F5007F81BF024AD36C5D
:1095C00043F02003D36408BD0020024008B5FFF734
:1095D0009FFFB0F5007F81BF024AD36C43F01003B8
:1095E000D36408BD0020024008B500F0CFF800F0B9
:1095F000C5F800F0D3F8FFF78BFFB0F5007F07D96F
:10960000FFF7C8FFFFF7D4FFBDE80840FFF7DEBF54
:1096100008BD000038B5064DEC68FFF779FFB0F5DE
:10962000007F84BFE86C044304F0350038BD00BF00
:109630000020024038B504460D4600F0B7F8FFF7A9
:1096400067FFB0F5007F124B17D9124A944214D924
:109650001A6D42F001021A65258000F0A7F8FFF7A5
:1096600057FFB0F5007F0A4B0CD90A4A944209D93A
:109670001A6D22F001021A6538BD1A6942F0010222
:109680001A61E9E71A6922F001021A61F4E700BFE2
:1096900000200240FFFF070810B5044600F086F8DE
:1096A000FFF736FFB0F5007F164B1BD9164A9442E0
:1096B00018D91A6D42F002021A655C651A6D42F003
:1096C00040021A6500F072F8FFF722FFB0F5007F44
:1096D0000C4B11D90C4A94420ED91A6D22F0020299
:1096E0001A6510BD1A6942F002021A615C611A69BA
:1096F00042F040021A61E5E71A6922F002021A619B
:10970000EFE700BF00200240FFFF070810B5104C34
:1097100000F04CF8236943F004032361236943F00C
:109720004003236100F042F8236923F0040323611E
:10973000236D43F004032365236D43F04003236549
:1097400000F034F8236D23F00403236510BD00BF3F
:1097500000200240034B044A5A6002F188325A60EA
:10976000704700BF0020024023016745024A136989
:1097700043F080031361704700200240024AD3681F
:1097800043F02003D360704700200240024AD368B0
:1097900043F00403D360704700200240024AD368BC
:1097A00043F01003D36070470020024008B5FFF774
:1097B00031FFC307FBD408BD38B505460C4689B256
:1097C000FFF738FF210CA81CBDE83840FFF732BF77
:1097D00010B50B4CFFF7EAFF23699B0501D400F09D
:1097E00027FA236943F020032361236943F04003F0
:1097F0002361FFF7DBFF236923F02003236110BD02
:109800000020024070B50B4C05460E46FFF7CEFF18
:1098100023699B0501D400F00BFA236943F0100380
:1098200023612E80FFF7C2FF236923F01003236119
:1098300070BD00BF002002402DE9F04100264FF02E
:109840000F0E9C46036847684CFA06F4E4071BD5E4
:10985000072E94BF9846B846B4B24FEA84048ABF34
:10986000203CA4B2A4B20EFA04F528EA0508A51C0F
:10987000ADB202FA05F501FA04F42C4344EA0804F7
:10988000072E94BF234627460136102EDCD10360F5
:109890004760BDE8F0810000024B084340F08000C3
:1098A0001860704700000140034A536823F0E063EA
:1098B0000B4303435360704700000140024AD369E1
:1098C0000343D361704700BF00000140016170474E
:1098D000090401617047806808407047C36801EA65
:1098E000030221EA030141EA0241016170478068F5
:1098F00080B27047C160704741F4803383618161F9
:10990000836183698369704703680B430360704711
:10991000036823EA01030360704703681943016089
:109920007047036823EA010303607047012243097B
:1099300003F1804303F50433196800F01F0002FAB5
:1099400000F00843186070470121430903F1804388
:1099500003F504331A6800F01F0001FA00F022EA50
:109960000000186070470122430903F1804303F5AA
:109970000433196800F01F0002FA00F00143196077
:109980001A6822EA000018607047FFF7CFBFFFF7A0
:10999000DBBF0000034A536823F0706343EA0063AF
:1099A0005360704700100240032802D0052806D0FB
:1099B0007047064A136843F4802313607047034AD4
:1099C000136A43F004031362704700BF00100240A3
:1099D000032802D0052806D07047064A136823F4EE
:1099E000802313607047034A136A23F00403136251
:1099F000704700BF00100240064A074B90421B68A8
:109A000004BF064B1B6803EB5103B3FBF1F3836008
:109A1000704700BF00380140C0090020C409002081
:109A2000C36808290CBF23F4805343F48053C360F8
:109A30007047036923F440530B4303617047C368C5
:109A400023F4C0630B43C3607047C36823F00C0367
:109A50000B43C3607047436923F440730B43436176
:109A60007047C36843F40053C3607047C36823F46E
:109A70000053C360704738B504460D4600F049F8FE
:109A800029462046BDE8384000F03BB810B50446F2
:109A900000F043F82046BDE8104000F036B84369B6
:109AA00043F0400343617047436923F0400343613F
:109AB0007047436943F0800343617047436923F073
:109AC000800343617047C36843F02003C36070475D
:109AD000C36823F02003C3607047C36843F080036A
:109AE000C3607047C36823F08003C3607047436955
:109AF00043F0010343617047436923F0010343616D
:109B00007047C1F30801416070474068C0F3080026
:109B1000704703681B06FCD5704703689B06FCD59D
:109B2000704703680B4214BF012000207047FEE716
:109B30007047000038B51A4A1A4B1B498B421AD39A
:109B400000211A4A93421BD34FF0E022D2F8143D71
:109B5000174C43F40073174DC2F8143DAC4212D3B6
:109B6000154C164DAC4212D3F7F7A4FB144C154D0F
:109B7000AC4210D338BD52F8040B43F8040BDDE7B8
:109B800043F8041BDEE754F8043B9847E6E754F833
:109B9000043B9847E6E754F8043B9847E8E700BFE2
:109BA000E0C5000800000020C80900204C0A002081
:109BB000D8C50008D8C50008D8C50008D8C5000811
:109BC000D8C50008D8C500084FF0E023014AC3F803
:109BD0000C2DFEE70100FA054FF0E023014AC3F81F
:109BE0000C2DFEE70400FA054FF0E02340F0BF60C3
:109BF00040F40030C3F80C0D70470000024A1368AF
:109C000043F010031360704700200240024A1368BB
:109C100023F010031360704700200240034A1368CA
:109C200023F0070303431360704700BF0020024086
:109C3000034B044A9A6002F188329A60704700BF71
:109C4000002002402301674506280AD8DFE800F01B
:109C5000040A0F14191E2300114A936843F4801359
:109C6000936070470E4A936843F40013F8E70C4A78
:109C7000936843F48003F3E7094A936843F40023AD
:109C8000EEE7074A936843F48023E9E7044A9368C0
:109C900043F40033E4E7024A936843F48033DFE798
:109CA0000010024006280AD8DFE800F0040A0F146A
:109CB000191E2300114A936843F480539360704740
:109CC0000E4A936843F40053F8E70C4A936843F450
:109CD0008043F3E7094A936843F40063EEE7074AD9
:109CE000936843F48063E9E7044A936843F400739C
:109CF000E4E7024A936843F48073DFE70010024010
:109D000006280AD8DFE800F0040A0F14191E230001
:109D1000114A936823F48053936070470E4A936806
:109D200023F40053F8E70C4A936823F48043F3E7E5
:109D3000094A936823F40063EEE7074A936823F423
:109D40008063E9E7044A936823F40073E4E7024A76
:109D5000936823F48073DFE70010024008B5134BCB
:109D6000062821D8DFE800F004080C1014181C00A5
:109D70009868C0F3001008BD9868C0F34010FAE777
:109D80009868C0F38010F6E79868C0F3C000F2E767
:109D90009868C0F38000EEE79868C0F34000EAE7F7
:109DA000986800F00100E6E700F0AEFB001002400A
:109DB000024A936843F40003936070470010024026
:109DC000024B9868C0F3C010704700BF00100240FB
:109DD000062824D8DFE800F004090E13181D20001F
:109DE000104B1868C0F3406070470E4B1868C0F302
:109DF000C06070470B4B1868C0F340707047094B48
:109E00001868C0F340407047064B1868C0F3400024
:109E10007047044B186AF9E7024B586AF6E70020CE
:109E2000704700BF00100240024608B51046FFF719
:109E3000CFFF0028FAD008BD06282AD8DFE800F0B6
:109E4000040A0F14191E2400124A136843F0807389
:109E5000136070470F4A136843F08063F8E70D4AB8
:109E6000136843F08053F3E70A4A136843F48033DE
:109E7000EEE7084A136843F00103E9E7054A136A6D
:109E800043F0010313627047024A536A43F001032F
:109E9000536270470010024006282AD8DFE800F01D
:109EA000040A0F14191E2400124A136823F0807349
:109EB000136070470F4A136823F08063F8E70D4A78
:109EC000136823F08053F3E70A4A136823F48033BE
:109ED000EEE7084A136823F00103E9E7054A136A2D
:109EE00023F0010313627047024A536A23F001030F
:109EF0005362704700100240024A136843F4002383
:109F00001360704700100240024A136823F40023D4
:109F10001360704700100240034A536823F00303A4
:109F200003435360704700BF00100240034A536868
:109F300023F4701343EA80435360704700100240DB
:109F4000034AD36A23F4706343EA0023D362704761
:109F500000100240034AD36A23F4704343EA0033FB
:109F6000D362704700100240034A536823F48033E1
:109F700043EA00435360704700100240034A5368AD
:109F800023F4003343EA404353607047001002401B
:109F9000024B186A00F40040704700BF00100240F6
:109FA000024A136A43F400431362704700100240F0
:109FB00006283BD8DFE800F0353535253504150097
:109FC0001B4B1A6A42F001021A621A6A9007FCD50A
:109FD0001A6A22F440721A621A6A42F480721A6291
:109FE0007047134B5A6A42F001025A625A6A91074B
:109FF000FCD51A6A22F440721A621A6A42F400729C
:10A00000EDE70B4B1A6842F480321A601A6892032B
:10A01000FCD51A6A22F440721A621A6A42F440723B
:10A02000DDE7034A136A23F440731362704700BFED
:10A0300000100240034A536823F4404343EA80334C
:10A040005360704700100240034A536823F4605382
:10A0500043EAC0235360704700100240034A53682C
:10A0600023F4E06343EA002353607047001002408A
:10A07000034A536823F0F00343EA00135360704728
:10A0800000100240044B5A6818B142F480025A6032
:10A09000704722F48002FAE700100240034AD36AB4
:10A0A00023F00F030343D362704700BF0010024048
:10A0B000034AD36A23F0F00343EA0013D3627047E4
:10A0C00000100240044BDA6A18B142F48032DA62BE
:10A0D000704722F48032FAE700100240024B5868C1
:10A0E000C0F38100704700BF0010024008B5042093
:10A0F000FFF7A2FEFFF798FE0020FFF70DFFFFF726
:10A10000B7FF0320FFF796FF0420FFF7A7FF00200B
:10A11000FFF79AFF0220FFF781FD0E20FFF706FFF1
:10A120000020FFF721FFFFF787FEFFF77DFE0220EB
:10A13000FFF7F2FE044B054A05491360054A11601A
:10A14000054A136008BD00BF0090D003BC09002081
:10A150000048E801C0090020C409002008B5042017
:10A16000FFF76AFEFFF760FE0020FFF7D5FEFFF75E
:10A170007FFF0320FFF75EFF0420FFF76FFF002043
:10A18000FFF762FF0E4A0120536843F480035360D7
:10A19000FFF744FD0A20FFF7C9FE0020FFF7E4FEA9
:10A1A000FFF74AFEFFF740FE0220FFF7B5FE054B22
:10A1B000054A06491360064A1160064A136008BD45
:10A1C00000100240006CDC02BC09002000366E0169
:10A1D000C0090020C409002008B50420FFF72CFEA8
:10A1E000FFF722FE0020FFF797FEFFF741FFFFF782
:10A1F00021FFFFF733FFFFF727FFFFF70FFD0420D5
:10A20000FFF794FE0020FFF7AFFEFFF715FEFFF704
:10A210000BFE0220FFF780FE034B044A1360044A42
:10A220001360044A136008BD00366E01BC090020AB
:10A23000C0090020C409002008B50420FFF7FCFD78
:10A24000FFF7F2FD0020FFF767FE0320FFF7F4FDA4
:10A25000FFF7EAFD0120FFF75FFE0020FFF708FF90
:10A26000FFF7E8FEFFF7FAFEFFF7EEFEFFF7D6FC7A
:10A270000120FFF75BFEFFF777FE0020FFF77EFE71
:10A28000FFF7DAFDFFF7D0FD0220FFF745FE044B94
:10A29000044A1360044A1360044A136008BD00BFF7
:10A2A00000366E01BC090020C0090020C40900204E
:10A2B00008B50420FFF7C0FDFFF7B6FD0020FFF74B
:10A2C0002BFE0320FFF7B8FDFFF7AEFD0120FFF7DF
:10A2D00023FE0020FFF7CCFE0320FFF7ABFE042097
:10A2E000FFF7BCFE0020FFF7AFFE0220FFF796FC51
:10A2F0000720FFF71BFE0120FFF736FE0020FFF7C7
:10A300003DFEFFF799FDFFF78FFD0220FFF704FEEA
:10A31000044B054A05491360054A1160054A13605C
:10A3200008BD00BF00A24A04BC090020005125025C
:10A33000C0090020C409002008B50420FFF77CFDF7
:10A34000FFF772FD0020FFF7E7FD0320FFF774FD24
:10A35000FFF76AFD0120FFF7DFFD0020FFF788FE11
:10A360000220FFF767FE0420FFF778FE0020FFF7CA
:10A370006BFE0220FFF752FC0420FFF7D7FD0120FF
:10A38000FFF7F2FD0020FFF7F9FDFFF755FDFFF79E
:10A390004BFD0220FFF7C0FD044B054A0549136041
:10A3A000054A1160054A136008BD00BF00A24A04B7
:10A3B000BC09002000512502C0090020C40900206A
:10A3C00008B50420FFF738FDFFF72EFD0020FFF74A
:10A3D000A3FD0320FFF730FDFFF726FD0120FFF767
:10A3E0009BFD0020FFF744FE0220FFF723FE042020
:10A3F000FFF734FE0020FFF727FE0220FFF70EFCD8
:10A400000720FFF793FD0120FFF7AEFDFFF7B6FD34
:10A410000020FFF711FDFFF707FD0220FFF77CFD8D
:10A42000044B054A05491360054A1160054A13604B
:10A4300008BD00BF00A24A04BC090020005125024B
:10A44000C0090020C409002008B50320FFF7F4FC70
:10A45000FFF7EAFC0120FFF75FFD0220FFF7DEFBBC
:10A460000020FFF705FE0220FFF7E4FD0420FFF7C0
:10A47000F5FD0020FFF7E8FD0420FFF719FE062098
:10A48000FFF75EFD0120FFF7D7FCFFF7CDFC0020B2
:10A49000FFF774FD104A0420D36A104943F4803357
:10A4A000D362FFF7FBFD0720FFF740FD0120FFF718
:10A4B0005BFD0020FFF7E6FDFFF7BEFCFFF7B4FCF5
:10A4C0000220FFF729FD064B064A1360064A116079
:10A4D000064A136008BD00BF00100240005125026B
:10A4E00000A24A04BC090020C0090020C4090020C1
:10A4F000044B1A6A42F480321A621A6A22F48032D9
:10A500001A62704700100240FEE708B5FFF7FCFF33
:10A5100041524D00756E6B6E6F776E004350552043
:10A52000696E666F726D6174696F6E3A0D002D20F1
:10A5300043505549443A2030782530386C780D0A1C
:10A54000002D20696D706C656D656E7465723A20C2
:10A5500025732028307825303278290D0A002D20E7
:10A560006172636869746563747572653A2000414D
:10A57000524D76362D4D0041524D76372D4D0020EF
:10A580002830782578290D0A002D207061727420FA
:10A590006E756D6265723A2000436F727465782D36
:10A5A0004D302B00436F727465782D4D3000436F32
:10A5B000727465782D4D3300436F727465782D4D3C
:10A5C0003400436F727465782D4D37002028307841
:10A5D00025303378290D0A002D2076617269616E6D
:10A5E000743A2025750D0A002D207265766973690D
:10A5F0006F6E3A2025750D0A00796573006E6F0045
:10A60000636865636B696E67206572726174613A35
:10A610002061636365737320746F2064656275677E
:10A620002072656769737465720D002D204D435566
:10A6300020494420636F64653A2030782530386CB7
:10A640007820284445565F49443D3078253033789A
:10A65000205245565F49443D307825303478290DE5
:10A660000A002D20646562756720617474616368F7
:10A6700065643A2025730D0A002D206465627567B4
:10A6800020686173206265656E206174746163681F
:10A6900065642C20627574204D4355204944206325
:10A6A0006F6465206973206E6F74207265616461E8
:10A6B000626C652C20617320646F63756D656E74C8
:10A6C000656420696E2074686520657272617461CA
:10A6D0000D002D2064656275672069732F686173B2
:10A6E000206265656E2061747461636865642C2006
:10A6F000627574204D435520494420636F64652082
:10A700006973207374696C6C206E6F74207265615C
:10A710006461626C652C20746869732069732061C0
:10A720006E20756E6B6E6F776E20626568617669FC
:10A730006F75720D002D2064656275672069732046
:10A7400061747461636865642C20616E64204D439C
:10A750005520494420636F6465206973206E6F77CC
:10A76000207265616461626C652E2044657461636A
:10A770006820646562756720284A5441472F535703
:10A78000442920746F2062652061626C6520746FBB
:10A7900020766572696679206572726174612069DC
:10A7A000737375650D002D2064656275672069738C
:10A7B000206E6F742061747461636865642C20611D
:10A7C0006E64204D435520494420636F64652069C1
:10A7D00073206E6F74207265616461626C652C20F9
:10A7E000617320646F63756D656E74656420696E56
:10A7F00020746865206572726174610D002D20649B
:10A8000065627567206973206E6F7420617474616E
:10A81000636865642C20627574204D43552049445B
:10A8200020636F6465206973207265616461626C86
:10A8300065202D3E2074686973206973206E6F74E3
:10A8400020616E2053544D33320D004A4550313053
:10A85000362049443A200053544D0047696761440B
:10A8600065766963650069566976697479002028A0
:10A87000636F6E742E3D25752C2049443D3078253C
:10A88000303278292C20706172743D307825303355
:10A89000780D0A00696E61636365737369626C6544
:10A8A0000074657374696E672061636365737369AF
:10A8B00062696C697479206F662061646472657383
:10A8C00073207370616365202874616B6573203237
:10A8D000206D696E75746573293A0D002D203078EE
:10A8E0002530386C782D30782530386C783A202532
:10A8F000730D0A002D206E6F206D61746368696EA0
:10A9000067206D656D6F7279206D617020666F755F
:10A910006E642E20706C656173652073656E6420B3
:10A92000636869702064657461696C732028707253
:10A9300065737320612920746F2066313033696438
:10A94000406375766F6F646F6F2E696E666F0D0072
:10A950002D206D656D6F7279206D6170206D617451
:10A96000636865732025730D0A006D616E756661FD
:10A970006374757265723A200053544D6963726F47
:10A98000656C656374726F6E69637300474400435E
:10A990004B53004368696E61204B6579205379738E
:10A9A00074656D0041504D004170656D69780048D7
:10A9B0004B0048616E677368756E003F3F3F005201
:10A9C0004F4D207461626C6520656E7472696573A9
:10A9D0003A0D002D2030782530386C7820282573EA
:10A9E000293A2030782530386C780D0A0064657675
:10A9F00069636520756E697175652049443A202543
:10AA000030386C782530386C782530346C782530C7
:10AA1000346C780D0A00636869702066616D696C3A
:10AA200079200028504944525F504152544E4F3DC6
:10AA3000307825303378293A2000284445565F493C
:10AA4000443D307825303378293A20006E6F7420E9
:10AA50007265616461626C652C2072657472792024
:10AA600077697468206465627567206174746163D6
:10AA7000686564006572726F6E656F7573207265CC
:10AA80006164696E672C2072656164206F766572FF
:10AA90002064656275672066697273740053544D53
:10AAA000333246313078206C6F772D64656E736970
:10AAB00074790053544D333246313078206D6564DB
:10AAC00069756D2D64656E736974790053544D33E7
:10AAD000324631307820686967682D64656E736925
:10AAE00074790053544D33324631307820584C2D10
:10AAF00064656E736974790053544D333246313056
:10AB00007820636F6E6E656374697669747900533B
:10AB1000544D3332463033780053544D333246303F
:10AB200034780053544D3332463035780053544D09
:10AB30003332463037780053544D3332463039780B
:10AB400000473037312F3038310053544D333247BE
:10AB500030373178782F53544D333247303831788D
:10AB60007800473033312F3034310053544D333275
:10AB70004730333178782F53544D333247303431A6
:10AB8000787800463430352F3430372F3431352F34
:10AB90003431370053544D3332463430352F53540B
:10ABA0004D3332463430372F53544D3332463431DF
:10ABB000352F53544D3332463431370046343278D2
:10ABC0002F3433780053544D3332463432782F5378
:10ABD000544D3332463433780046343031005354C8
:10ABE0004D33324634303178422F430053544D3385
:10ABF000324634303178442F4500463431310053E9
:10AC0000544D33324634313178432F45004631308C
:10AC1000300053544D333246313030206C6F772F33
:10AC20006D656469756D2D64656E73697479005323
:10AC3000544D33324631303020686967682D646581
:10AC40006E736974790041504D333246313078006B
:10AC500063686970207265766973696F6E20285227
:10AC600045565F49443D307825303478293A2000F4
:10AC7000312F322F332F582F5900412F3100746F4D
:10AC800020676574206368697020726576697369EE
:10AC90006F6E20696E666F726D6174696F6E2C20C5
:10ACA0006174746163682064656275670D00746522
:10ACB0007374696E672070696E7320746F206669A3
:10ACC00067757265206F75742076617269616E7444
:10ACD000202870696E73207469656420746F206722
:10ACE000726F756E642063616E206C6561642074A0
:10ACF0006F2066616C736520706F73697469766527
:10AD000073293A0D002D20746869732069732070CF
:10AD1000696E20636F756E742076617269616E74FE
:10AD20002025632C20776974682025752070696E52
:10AD3000730D0A002D2074686973206973206E6F8B
:10AD4000742070696E20636F756E7420766172690D
:10AD5000616E742025632C20776974682025752026
:10AD600070696E730D0A002D20636F756C64206E20
:10AD70006F74206964656E74696679206E756D62A2
:10AD80006572206F662070696E733A207468652062
:10AD900070696E6F757420697320756E6B6E6F7756
:10ADA0006E0D006D697373696E670070726573650F
:10ADB0006E7400616273656E740074657374696E9D
:10ADC00067207065726970686572616C2070726569
:10ADD00073656E63653A0D002D2025733A20257347
:10ADE0000D0A0073797374656D206D656D6F7279EE
:10ADF0003A200053544D333220626F6F746C6F6190
:10AE00006465722076322E32004744333220626FFE
:10AE10006F746C6F616465722076312E3000415022
:10AE20004D333220626F6F746C6F6164657220768F
:10AE3000322E3200484B333220626F6F746C6F6178
:10AE40006465722076322E3200756E6B6E6F776E8F
:10AE500020626F6F746C6F616465720020284352CA
:10AE6000433D30782530386C782900666C61736812
:10AE70002026205352414D2073697A6520696E6601
:10AE80006F726D6174696F6E202863616E207461EA
:10AE90006B652032206D696E75746573293A0D00FB
:10AEA0002D206164766572746973656420666C61D7
:10AEB00073682073697A653A2000756E6B6E6F77E0
:10AEC0006E202870726F6261626C79206120636FFE
:10AED000756E746572666569742F64656665637402
:10AEE000697665206D6963726F2D636F6E74726F22
:10AEF0006C6C65720D002575204B420D0A002D20EB
:10AF00007265616461626C6520666C617368207350
:10AF1000697A653A20256C752062797465732028FA
:10AF2000256C75204B42290D0A002D206F76657225
:10AF300020616476657274697365642077726974E0
:10AF400061626C6520666C6173682073697A653A2A
:10AF500020256C752062797465732028256C752016
:10AF60004B42290D0A002D207265616461626C6597
:10AF7000205352414D3A20256C75206279746573D7
:10AF80002028256C75204B42290D0A002D20777250
:10AF9000697461626C65205352414D3A20256C758D
:10AFA0002062797465732028256C75204B42290D29
:10AFB0000A006964656E74696679696E67204D433D
:10AFC00055202863616E2074616B652032206D69A5
:10AFD0006E75746573293A20002573333225730D1D
:10AFE0000A00257333322573256325630D0A000D8E
:10AFF0000A4375566F6F646F6F2046313033204DB2
:10B000004355206964656E7469666965720D0073E5
:10B0100074617274696E6720656D626564646564ED
:10B02000205541525420626F6F746C6F6164657279
:10B030000D006964656E7469666965722076657273
:10B0400073696F6E3A2025750D0A00616C6C20647F
:10B050006F6E650D00617661696C61626C6520637D
:10B060006F6D6D616E64733A0D006820202020734F
:10B07000686F7720746869732068656C700D006272
:10B0800020202020737461727420656D6265646491
:10B090006564205541525420626F6F746C6F616417
:10B0A00065720D0072202020207265736574204D3A
:10B0B00043552028652E672E207265737461727463
:10B0C000206170706C69636174696F6E290D007620
:10B0D0002020202073686F77206964656E7469662C
:10B0E0006965722076657273696F6E0D006120204C
:10B0F000202073686F7720616C6C20696E666F72B8
:10B100006D6174696F6E0D006D2020202073686F73
:10B1100077206D616E7566616374757265720D007E
:10B12000662020202073686F77204D43552066618C
:10B130006D696C790D00732020202073686F772073
:10B14000666C61736820616E64205352414D2073B8
:10B15000697A650D00632020202073686F77204393
:10B1600050550D00752020202073686F77204D43C7
:10B170005520756E697175652049440D006A20205F
:10B18000202073686F77204A45503130362049447B
:10B190000D00742020202073686F7720524F4D20BF
:10B1A0007461626C650D00792020202073686F77D0
:10B1B0002073797374656D206D656D6F72790D0004
:10B1C00069202020206964656E74696679204D438A
:10B1D00055206D6F64656C0D007020202020746513
:10B1E0007374207065726970686572616C730D00AC
:10B1F0006E20202020746573742070696E20636F48
:10B20000756E740D006C20202020746573742061AD
:10B2100063636573736962696C697479206F662012
:10B22000616464726573732073706163650D00659A
:10B230002020202074657374206572726174610D22
:10B24000000D0A746F207375626D697420697373E1
:10B25000756573206F7220756E6B6E6F776E2064EC
:10B2600065766963652064657461696C732C20730D
:10B27000656E6420616C6C20696E666F726D6174BE
:10B28000696F6E2028707265737320612920746F56
:10B2900020663130336964406375766F6F646F6F19
:10B2A0002E696E666F0D007265626F6F74696E67EE
:10B2B0000D00756E6B6E6F776E20636F6D6D616ED6
:10B2C000642E2074797065206820666F722068652E
:10B2D0006C700D004631303043340046313030431D
:10B2E000360046313030433800463130304342007A
:10B2F000463130305234004631303052360046311B
:10B30000303052380046313030524200463130330E
:10B3100054380046313033544200463130334342D2
:10B320000046313033523800463130335242004605
:10B330003130335638004631303356420047504999
:10B340004F42004750494F43004750494F44004740
:10B3500050494F45004750494F46004750494F47D5
:10B360000054494D310054494D320054494D330089
:10B3700054494D340054494D350054494D3600541C
:10B38000494D370054494D380054494D313500542A
:10B39000494D31360054494D3137005553415254CF
:10B3A00032005553415254330053504931005350E9
:10B3B0004932004932433100493243320043454368
:10B3C000005553420043414E310043414E32005339
:10B3D000544D333246313033437800434B5333328C
:10B3E00046313033433800474433324631303343FB
:10B3F000380041504D333246313033433800484BEA
:10B40000333246313033433800524F4D53435300AB
:10B41000524F4D44575400524F4D46504200524FE8
:10B420004D49544D00524F4D5450495500524F4DC7
:10B4300045544D004D454D545950450050494434F4
:10B4400000504944350050494436005049443700C3
:10B450005049443000504944310050494432005072
:10B46000494433004349443000434944310043498F
:10B47000443200434944330003030000000C014000
:10B4800088B4000807000000000100020004000862
:10B4900000100020004000000403000000100140E4
:10B4A000B8B400080C0000000503000000140140BF
:10B4B000D0B40008010000000100020004001000E8
:10B4C000200040008000000100020004000800107D
:10B4D0000400000003030000000C0140E4B4000875
:10B4E00001000000010000000503000000140140FD
:10B4F00008B500080D000000060300000018014018
:10B5000022B50008100000000800100020004000D4
:10B51000800000010002000400080010002000402C
:10B52000008001000200040008001000200040001C
:10B53000800000010002000400080010002000400C
:10B540000080000007030000001C014064B50008F3
:10B550000500000008030000002001406EB500084F
:10B5600010000000000800100020004000800100D2
:10B5700002000400080010002000400080000001CC
:10B5800000020004000800100020004000800000BD
:10B59000CFB3000814C0000820000000DBB300088F
:10B5A000B0BA000839000000E7B300085CBD00082D
:10B5B0001C000000F2B3000818B9000822000000C7
:10B5C000FEB30008ACBE00081E000000D4B20008A4
:10B5D0001004300054B80008DBB20008200430002A
:10B5E00054B80008E2B20008400830006FB8000804
:10B5F000E9B20008800830006FB80008F0B2000817
:10B600001004400054B80008F7B2000820044000BD
:10B6100054B80008FEB20008400840006FB80008A7
:10B6200005B30008800840006FB800080CB300089C
:10B6300040142400A5B8000813B3000880142400A7
:10B64000A5B80008EBB30008401430008AB8000821
:10B650001AB30008801430008AB8000821B300082B
:10B66000401440008AB8000828B300088014400045
:10B670008AB800082FB30008401464008AB8000894
:10B6800036B30008801464008AB80008EBB30008E1
:10B6900040143000C0B800081AB30008801430000D
:10B6A000C0B800083DB30008030383010C0C01403F
:10B6B0000100000043B30008040384010C100140A2
:10B6C0000100000049B30008050385010C14014086
:10B6D000010000004FB30008060386010C1801406A
:10B6E0000100000055B30008070387010C1C01404E
:10B6F000010000005BB30008080388010C20014032
:10B700000100000061B300080B038B01242C0140F1
:10B710000100000066B3000880030002240000401E
:10B72000010000006BB30008810301022404004003
:10B730000100000070B300088203020224080040E8
:10B740000100000075B3000883030302240C0040CD
:10B75000010000007AB300088403040224100040B2
:10B76000010000007FB30008850305022414004097
:10B770000100000084B300080D038D012434014052
:10B780000100000089B3000810039001244001402B
:10B79000010000008FB3000811039101244401400F
:10B7A0000100000095B300081203920124480140F3
:10B7B000010000009BB300089103110208440040FF
:10B7C00001000000A2B300089203120208480040E2
:10B7D00001000000A9B300080C038C0110300140E7
:10B7E00008000000AEB300088E030E0210380040BF
:10B7F00008000000B3B30008950315020854004088
:10B8000001000000B8B30008960316020858004073
:10B8100001000000BDB300089E031E020478004032
:10B8200001000000C1B30008970317024C5C004000
:10B8300001000000C5B3000899031902006400402C
:10B8400010000000CAB300089A031A020068004002
:10B8500010000000010100000000010101000100D2
:10B8600000000101010100010001000100000001D0
:10B8700001000000000101010101000000010101BF
:10B8800001010101010101000000010101010000AD
:10B89000010101010000000000000001010101019F
:10B8A000010001010001010000000001010101008F
:10B8B0000000000000000100010001000001010083
:10B8C0000101010000000101010100000000000071
:10B8D0000001010101010100000100005A90000077
:10B8E00044B500080200000056640000E8B40008F7
:10B8F000020000005240000098B40008020000005E
:10B900004330000078B40008010000005424000017
:10B91000D4B400080100000000000000FFFF010097
:10B920000100000000000200FFFFFF070000000010
:10B9300000000008FFFF01080100000000000208ED
:10B94000FFEFFF1F0000000000F0FF1FFFFBFF1FC5
:10B950000100000000FCFF1FFFFFFF1F00000000B0
:10B9600000000020FF4F00200100000000500020D8
:10B97000FFFFFF210000000000000022FFFF09225E
:10B980000100000000000A22FFFFFF3F000000004E
:10B9900000000040FF7F01400100000000800140E6
:10B9A000FFFF01400000000000000240FF030240D2
:10B9B0000100000000040240FF0F024000000000F0
:10B9C00000100240FF13024001000000001402407A
:10B9D000FF2F02400000000000300240FF33024011
:10B9E0000100000000340240FF3F02400000000060
:10B9F00000400240FF4302400100000000440240BA
:10BA0000FFFFFF410000000000000042FFFF2F4247
:10BA10000100000000003042FFFF3F420000000034
:10BA200000004042FF7F4042010000000080404291
:10BA3000FFFF41420000000000004242FF7F4242FF
:10BA40000100000000804242FFFF4542000000006C
:10BA500000004642FF7F464201000000008046424F
:10BA6000FFFF47420000000000004842FF7F4842BD
:10BA70000100000000804842FFFFFF5F000000005F
:10BA800000000060FFFFFFAF01000000000000B0F9
:10BA9000FFFFFFDF00000000000000E0FFFF0FE0FD
:10BAA00001000000000010E0FFFFFFFF00000000A9
:10BAB00000000000FFFF0108010000000000020874
:10BAC000FFEFFF1F0000000000F0FF1FFFF9FF1F46
:10BAD0000100000000FAFF1FFFFFFF1F0000000031
:10BAE00000000020FF0B004001000000000C00409F
:10BAF000FF2700400000000000280040FF33004006
:10BB00000100000000340040FF370040000000004A
:10BB100000380040FF3B004001000000003C0040B6
:10BB2000FF4300400000000000440040FF4B004085
:10BB300001000000004C0040FF53004000000000E6
:10BB400000540040FF670040010000000068004012
:10BB5000FF6B004000000000006C0040FF730040DD
:10BB60000100000000740040FFFF004000000000E2
:10BB700000000140FF1B014001000000001C0140CB
:10BB8000FF2301400000000000240140FF3301407A
:10BB90000100000000340140FF37014000000000B8
:10BBA00000380140FF3B014001000000003C014023
:10BBB000FFFF01400000000000000240FF030240C0
:10BBC0000100000000040240FF0F024000000000DE
:10BBD00000100240FF130240010000000014024068
:10BBE000FF1F02400000000000200240FF2302402F
:10BBF0000100000000240240FF2F0240000000006E
:10BC000000300240FF3302400100000000340240D7
:10BC1000FFFFFF410000000000000042FF7F0142E3
:10BC20000100000000800142FFFF0442000000000C
:10BC300000000542FF7F064201000000008006422E
:10BC4000FFFF06420000000000000742FF7F07429E
:10BC50000100000000800742FF7F08420000000052
:10BC600000800842FF7F0942010000000080094275
:10BC7000FF7F0A420000000000800A42FFFF0C42E2
:10BC80000100000000000D42FF7F0D420000000097
:10BC900000800D42FF7F0E420100000000800E4236
:10BCA000FFFF1F420000000000002042FF7F2342F0
:10BCB0000100000000802342FF7F244200000000BA
:10BCC00000802442FF7F26420100000000802642BF
:10BCD000FFFF26420000000000002742FF7F2742AE
:10BCE0000100000000802742FFFF3F4200000000EB
:10BCF00000004042FF7F40420100000000804042BF
:10BD0000FFFF41420000000000004242FF7F42422C
:10BD10000100000000804242FFFF4342000000009B
:10BD200000004442FF7F4442010000000080444282
:10BD3000FFFF45420000000000004642FF7F4642F0
:10BD40000100000000804642FF0F00A0000000003C
:10BD5000001000A0FFFFFFFF010000000000000036
:10BD6000FF4F00200100000000500020FFFFFF21D6
:10BD70000000000000000022FFFF09220100000077
:10BD800000000A22FFFFFF3F00000000000000400B
:10BD9000FF7F01400100000000800140FFFF0140E3
:10BDA0000000000000000240FF030240010000000C
:10BDB00000040240FF0F024000000000001002409B
:10BDC000FF1302400100000000140240FF1F024068
:10BDD0000000000000200240FF230240010000009C
:10BDE00000240240FF2F024000000000003002400B
:10BDF000FF3302400100000000340240FFFFFF411A
:10BE00000000000000000042FFFF2F420100000080
:10BE100000003042FFFF3F420000000000004042AF
:10BE2000FF7F40420100000000804042FFFF41428E
:10BE30000000000000004242FF7F4242010000007B
:10BE400000804242FFFF43420000000000004442E5
:10BE5000FF7F44420100000000804442FFFF454252
:10BE60000000000000004642FF7F46420100000043
:10BE700000804642FFFFFF5F0000000000000060FE
:10BE8000FF0F00A001000000001000A0FFFFFFDF77
:10BE900000000000000000E0FFFF0FE001000000D4
:10BEA000000010E0FFFFFFFF0000000000000000A6
:10BEB000FF4F00200100000000500020FFFFFF2185
:10BEC0000000000000000022FFFF09220100000026
:10BED00000000A22FFFFFF3F0000000000000040BA
:10BEE000FF7F01400100000000800140FFFF014092
:10BEF0000000000000000240FF03024001000000BB
:10BF000000040240FF0F0240000000000010024049
:10BF1000FF1302400100000000140240FF1F024016
:10BF20000000000000200240FF230240010000004A
:10BF300000240240FF2F02400000000000300240B9
:10BF4000FF3302400100000000340240FFFF0240C6
:10BF50000000000000000340FF0303400100000058
:10BF600000040340FFFFFF4100000000000000420A
:10BF7000FFFF2F420100000000003042FFFF3F4260
:10BF80000000000000004042FF7F4042010000002E
:10BF900000804042FFFF414200000000000042429A
:10BFA000FF7F42420100000000804242FFFF434207
:10BFB0000000000000004442FF7F444201000000F6
:10BFC00000804442FFFF454200000000000046425E
:10BFD000FF7F46420100000000804642FFFF5F42B3
:10BFE0000000000000006042FF7F6042010000008E
:10BFF00000806042FFFFFFDF00000000000000E063
:10C00000FFFF0FE001000000000010E0FFFFFFFF56
:10C010000000000000000000FFFF01000100000020
:10C0200000000200FFFFFF07000000000000000802
:10C03000FFFF01080100000000000208FFEFFF1FE2
:10C040000000000000F0FF1FFFF9FF1F01000000CB
:10C0500000FAFF1FFFFFFF1F00000000000000208C
:10C06000FF4F00200100000000500020FFFFFF21D3
:10C070000000000000000022FFFF09220100000074
:10C0800000000A22FFFFFF3F000000000000004008
:10C09000FF7F00400100000000800040FFFF0040E3
:10C0A0000000000000000140FF3F014001000000CF
:10C0B00000400140FFFF014000000000000002407E
:10C0C000FF0302400100000000040240FF0F024095
:10C0D0000000000000100240FF13024001000000B9
:10C0E00000140240FF2F0240000000000030024018
:10C0F000FF3302400100000000340240FFFFFF4117
:10C100000000000000000042FFFF0F42010000009D
:10C1100000001042FFFF1F4200000000000020420C
:10C12000FFFF27420100000000002842FFFF3F42BE
:10C130000000000000004042FF7F4042010000007C
:10C1400000804042FFFF41420000000000004242E8
:10C15000FF7F42420100000000804242FFFF454253
:10C160000000000000004642FF7F46420100000040
:10C1700000804642FFFFFFDF00000000000000E0FB
:10C18000FFFF0FE001000000000010E0FFFFFFFFD5
:10C190000000000000F00FE009B4000804F00FE018
:10C1A00010B4000808F00FE017B400080CF00FE01E
:10C1B0001EB4000810F00FE025B4000814F00FE0E2
:10C1C0002DB40008CCFF0FE034B40008D0FF0FE01E
:10C1D0003CB40008D4FF0FE041B40008D8FF0FE0E2
:10C1E00046B40008DCFF0FE04BB40008E0FF0FE0AE
:10C1F00050B40008E4FF0FE055B40008E8FF0FE07A
:10C200005AB40008ECFF0FE05FB40008F0FF0FE045
:10C2100064B40008F4FF0FE069B40008F8FF0FE011
:10C220006EB40008FCFF0FE073B400081800002093
:10C230000A000000494E4600696E66004E414E00FD
:10C240006E616E00303132333435363738396162E1
:10C2500063646566000000003031323334353637B0
:10C26000383941424344454600000000286E756C51
:10C270006C290000300000002020202020202020F9
:10C28000202020202020202030303030303030302E
:10C2900030303030303030304E614E00496E66699B
:10C2A0006E6974790000000042616C6C6F632073EA
:10C2B0007563636565646564000000002E2E2F2E93
:10C2C0002E2F2E2E2F2E2E2F2E2E2F2E2E2F2E2E89
:10C2D0002F2E2E2F6E65776C69622D342E312E3005
:10C2E0002F6E65776C69622F6C6962632F7374645B
:10C2F0006C69622F64746F612E630000430000005C
:10C30000504F5349580000002E0000002E2E2F2EB3
:10C310002E2F2E2E2F2E2E2F2E2E2F2E2E2F2E2E38
:10C320002F2E2E2F6E65776C69622D342E312E30B4
:10C330002F6E65776C69622F6C6962632F7374640A
:10C340006C69622F6D707265632E630000000000DF
:10C350000080E03779C34143176E05B5B5B8934601
:10C36000F5F93FE9034F384D321D30F94877825ACD
:10C370003CBF737FDD4F1575000000000000F03FEB
:10C3800000000000000024400000000000005940B0
:10C390000000000000408F40000000000088C34003
:10C3A00000000000006AF8400000000080842E4178
:10C3B00000000000D01263410000000084D79741C4
:10C3C0000000000065CDCD41000000205FA00242CA
:10C3D000000000E876483742000000A2941A6D423F
:10C3E000000040E59C30A2420000901EC4BCD64232
:10C3F00000003426F56B0C430080E03779C34143DD
:10C4000000A0D8855734764300C84E676DC1AB4352
:10C41000003D9160E458E143408CB5781DAF154470
:10C4200050EFE2D6E41A4B4492D54D06CFF080444B
:10C43000F64AE1C7022DB544B49DD9794378EA4460
:10C44000BC89D897B2D29C3C33A7A8D523F64939EA
:10C450003DA7F444FD0FA5329D978CCF08BA5B250C
:10C46000436FAC642806C80A0500000019000000EC
:10C470007D000000202020202020202020202020BF
:10C4800020202020303030303030303030303030EC
:10C49000303030302C2066756E6374696F6E3A20D0
:10C4A00000000000617373657274696F6E2022254D
:10C4B0007322206661696C65643A2066696C652048
:10C4C000222573222C206C696E6520256425732536
:10C4D000730A00000020202020202020202028286F
:10C4E0002828282020202020202020202020202034
:10C4F0002020202020881010101010101010101074
:10C5000010101010100404040404040404040410A3
:10C510001010101010104141414141410101010131
:10C5200001010101010101010101010101010101FB
:10C530001010101010104242424242420202020207
:10C5400002020202020202020202020202020202CB
:10C55000101010102000000000000000000000007B
:10C5600000000000000000000000000000000000CB
:10C5700000000000000000000000000000000000BB
:10C5800000000000000000000000000000000000AB
:10C59000000000000000000000000000000000009B
:10C5A000000000000000000000000000000000008B
:10C5B000000000000000000000000000000000007B
:10C5C000000000000000000000000000000000006B
:08C5D000000000000000000063
:08C5D800C4CBFF7F010000004D
:10C5E00001000000BBA900083F000000BBA9000833
:10C5F0003F0000001800002000000000040300209D
:10C600006C030020D40300200000000000000000A4
:10C61000000000000000000000000000000000001A
:10C62000000000000000000000000000000000000A
:10C6300000000000000000000000000000000000FA
:10C6400000000000000000000000000000000000EA
:10C6500000000000000000000000000000000000DA
:10C6600000000000000000000000000000000000CA
:10C6700000000000000000000000000000000000BA
:10C6800000000000000000000000000000000000AA
:10C69000000000000000000000000000000000009A
:10C6A00001000000000000000E33CDAB34126DE637
:10C6B000ECDE05000B0000000000000000000000A0
:10C6C000000000000000000000000000000000006A
:10C6D000000000000000000000000000000000005A
:10C6E000000000000000000000000000000000004A
:10C6F000000000000000000000000000000000003A
:10CA200043000000000000000000000000000000C3
:10CA300000000000000000000000000000000000F6
:10CA400043000000000000000000000000000000A3
:10CA500000000000000000000000000000000000D6
:10CA60004300000000000000000000000000000083
:10CA700000000000000000000000000000000000B6
:10CA80004300000000000000000000000000000063
:10CA90000000000000000000000000000000000096
:10CAA0004300000000000000000000000000000043
:10CAB0000000000000000000000000000000000076
:10CAC0004300000000000000000000000000000023
:10CAD0000000000000000000000000000000000056
:10CAE0004300000000000000000000000000000003
:10CAF0000000000000000000000000000000000036
:10CB0000657D0008895B000800000000D4C40008AF
:10CB100008C30008A0C40008A0C40008A0C40008FE
:10CB2000A0C40008A0C40008A0C40008A0C4000855
:10CB3000A0C40008A0C40008FFFFFFFFFFFFFFFF25
:10CB4000FFFFFFFFFFFF0000010041534349490081
:10CB500000000000000000000000000000000000D5
:10CB6000000000000000000000004153434949005C
:10CB700000000000000000000000000000000000B5
:10CB800000000000000000000000000000000000A5
:10CB900000000000AC050020AC050020B40500201A
:10CBA000B4050020BC050020BC050020C405002001
:10CBB000C4050020CC050020CC050020D4050020B1
:10CBC000D4050020DC050020DC050020E405002061
:10CBD000E4050020EC050020EC050020F405002011
:10CBE000F4050020FC050020FC05002004060020C0
:10CBF000040600200C0600200C060020140600206D
:10CC0000140600201C0600201C060020240600201C
:10CC1000240600202C0600202C06002034060020CC
:10CC2000340600203C0600203C060020440600207C
:10CC3000440600204C0600204C060020540600202C
:10CC4000540600205C0600205C06002064060020DC
:10CC5000640600206C0600206C060020740600208C
:10CC6000740600207C0600207C060020840600203C
:10CC7000840600208C0600208C06002094060020EC
:10CC8000940600209C0600209C060020A40600209C
:10CC9000A4060020AC060020AC060020B40600204C
:10CCA000B4060020BC060020BC060020C4060020FC
:10CCB000C4060020CC060020CC060020D4060020AC
:10CCC000D4060020DC060020DC060020E40600205C
:10CCD000E4060020EC060020EC060020F40600200C
:10CCE000F4060020FC060020FC06002004070020BB
:10CCF000040700200C0700200C0700201407002068
:10CD0000140700201C0700201C0700202407002017
:10CD1000240700202C0700202C07002034070020C7
:10CD2000340700203C0700203C0700204407002077
:10CD3000440700204C0700204C0700205407002027
:10CD4000540700205C0700205C07002064070020D7
:10CD5000640700206C0700206C0700207407002087
:10CD6000740700207C0700207C0700208407002037
:10CD7000840700208C0700208C07002094070020E7
:10CD8000940700209C0700209C070020A407002097
:10CD9000A4070020AC070020AC070020B407002047
:10CDA000B4070020BC070020BC070020C4070020F7
:10CDB000C4070020CC070020CC070020D4070020A7
:10CDC000D4070020DC070020DC070020E407002057
:10CDD000E4070020EC070020EC070020F407002007
:10CDE000F4070020FC070020FC07002004080020B6
:10CDF000040800200C0800200C0800201408002063
:10CE0000140800201C0800201C0800202408002012
:10CE1000240800202C0800202C08002034080020C2
:10CE2000340800203C0800203C0800204408002072
:10CE3000440800204C0800204C0800205408002022
:10CE4000540800205C0800205C08002064080020D2
:10CE5000640800206C0800206C0800207408002082
:10CE6000740800207C0800207C0800208408002032
:10CE7000840800208C0800208C08002094080020E2
:10CE8000940800209C0800209C080020A408002092
:10CE9000A4080020AC080020AC080020B408002042
:10CEA000B4080020BC080020BC080020C4080020F2
:10CEB000C4080020CC080020CC080020D4080020A2
:10CEC000D4080020DC080020DC080020E408002052
:10CED000E4080020EC080020EC080020F408002002
:10CEE000F4080020FC080020FC08002004090020B1
:10CEF000040900200C0900200C090020140900205E
:10CF0000140900201C0900201C090020240900200D
:10CF1000240900202C0900202C09002034090020BD
:10CF2000340900203C0900203C090020440900206D
:10CF3000440900204C0900204C090020540900201D
:10CF4000540900205C0900205C09002064090020CD
:10CF5000640900206C0900206C090020740900207D
:10CF6000740900207C0900207C090020840900202D
:10CF7000840900208C0900208C09002094090020DD
:10CF8000940900209C0900209C090020A40900208D
:10CF9000A4090020FFFFFFFF0000020000127A003A
:08CFA00000127A0000127A0071
:0400000508009B351F
:00000001FF
